:06000000E5EF3BF01200E9
:08000800046ED8CF05F0E0CF33
:1000100006F00001E9CF0CF0EACF07F0E1CF08F0DD
:10002000E2CF09F0D9CF0AF0DACF0BF0F3CF12F01C
:10003000F4CF13F0FACF14F0F5CF15F0F6CF16F099
:10004000F7CF17F000C00EF001C00FF002C010F0A3
:1000500003C011F0F2AA30EF00F0F2B45DEF00F04F
:100060009DA036EF00F09EB036EF05F00EC000F018
:100070000FC001F010C002F011C003F00CC0E9FF86
:1000800007C0EAFF078E08C0E1FF09C0E2FF0AC00F
:10009000D9FF0BC0DAFF12C0F3FF13C0F4FF14C086
:1000A000FAFF15C0F5FF16C0F6FF17C0F7FF0450A2
:1000B00006C0E0FF05C0D8FF1000522AD8B4532A6A
:1000C000552A5550090802E2542A556A670ED76E20
:1000D000690ED66EF29436EF00F03C48544D4C3E1B
:1000E0003C424F44593E3C48313E34303420457206
:1000F000726F723C2F48313E3C48523E3C503E4667
:10010000696C65204E6F7420666F756E642E3C2F8F
:10011000424F44593E3C2F48544D4C3E00003C4811
:10012000544D4C3E3C424F44593E3C48313E3530A4
:1001300030204572726F723C2F48313E3C48523E2F
:100140003C503E496E7465726E616C2053657276E8
:100150006572204572726F723C2F424F44593E3C8B
:100160002F48544D4C3E0000485454502F312E30EF
:1001700020254C5520004E6F7420666F756E64000C
:10018000536572766572204572726F7200000D0AB7
:10019000436F6E74656E742D547970653A2000005B
:1001A000746578742F68746D6C000D0A0D0A000078
:1001B0000A3C48544D4C3E0A3C686561643E0A2046
:1001C000203C6C696E6B2072656C3D227374796C97
:1001D0006573686565742220687265663D2268747F
:1001E0007470733A2F2F636F64652E6A7175657230
:1001F000792E636F6D2F75692F312E31322E312F8D
:100200007468656D65732F626173652F6A717565BA
:1002100072792D75692E637373223E0A20203C7318
:100220006372697074207372633D226874747073B2
:100230003A2F2F636F64652E6A71756572792E632C
:100240006F6D2F6A71756572792D312E31322E34B2
:100250002E6A73223E3C2F7363726970743E0A20CB
:10026000203C736372697074207372633D226874FA
:100270007470733A2F2F636F64652E6A717565729F
:10028000792E636F6D2F75692F312E31322E312FFC
:100290006A71756572792D75692E6A73223E3C2FDD
:1002A0007363726970743E0A20203C7363726970D4
:1002B000743E24282066756E6374696F6E28292049
:1002C0007B2428202223612220292E6163636F7200
:1002D00064696F6E28293B207D20293B3C2F736386
:1002E000726970743E0A3C2F686561643E0A3C4244
:1002F0004F44593E0A3C6469762069643D2261227C
:100300003E0A3C68333E54656D7065726174757267
:10031000613C2F68333E0A3C6469763E3C68323E5D
:100320002532202623383435313B3C2F68323E3C81
:100330002F6469763E0A3C68333E4D696E207465D1
:100340006D70657261747572613C2F68333E0A3C52
:100350006469763E0A3C464F524D204D4554484F05
:10036000443D4745543E0A4D696E3C696E70757454
:1003700020747970653D227465787422206E616DF9
:10038000653D226D696E74656D222076616C7565C0
:100390003D222535222073697A653D322F3E262382
:1003A000383435313B0A3C494E505554205459504D
:1003B000453D227375626D6974222076616C7565A6
:1003C0003D225A617069737A223E0A3C2F464F5291
:1003D0004D3E0A3C2F6469763E0A3C68333E4465D4
:1003E00076313C2F68333E0A3C6469763E0A3C46CF
:1003F0004F524D204D4554484F443D4745543E0AC9
:100400003C494E50555420747970653D22726164A8
:10041000696F22206E616D653D2264657631222010
:1004200076616C75653D2231222025313E4F4E3C70
:1004300062722F3E2020200A3C494E5055542074B1
:100440007970653D22726164696F22206E616D650D
:100450003D2264657631222076616C75653D2230DF
:10046000222025303E4F46463C62722F3E0A3C49D0
:100470004E50555420545950453D227375626D6954
:1004800074222076616C75653D2255737461772204
:100490003E0A3C2F464F524D3E0A3C2F6469763E41
:1004A0000A3C68333E5A616C616E69653C2F683363
:1004B0003E0A3C6469763E5374616E2025363C2FBB
:1004C0006469763E0A3C68333E49503C2F68333EAF
:1004D0000A3C6469763E0A3C464F524D204D4554D5
:1004E000484F443D4745543E0A4950203139322E49
:1004F0003136382E302E3C696E70757420747970E8
:10050000653D227465787422206E616D653D2269B7
:1005100070222076616C75653D2225332220736937
:100520007A653D312F3E3C62722F3E0A4761746509
:10053000776179203139322E3136382E302E3C69B0
:100540006E70757420747970653D227465787422BC
:10055000206E616D653D2269706774222076616C42
:1005600075653D222534222073697A653D312F3E21
:100570003C62722F3E0A3C494E505554205459500B
:10058000453D227375626D6974222076616C7565D4
:100590003D225A617069737A223E0A3C2F464F52BF
:1005A0004D3E0A3C2F6469763E0A3C2F6469763ED4
:1005B0000A3C2F424F44593E3C2F48544D4C3E0A72
:1005C00000000A7B2264617461223A207B0A227453
:1005D000656D223A222532222C0A226D696E7465DD
:1005E0006D223A222535222C0A2264657631223A80
:1005F000222531222C0A227761746572223A222543
:1006000036220A7D7D0A0000636865636B656400BD
:10061000636865636B656400030E0301E25F11E3C9
:10062000030EEA6EE20EE96EFC0EEF16D890EF3282
:10063000EF32EF5006E0070E006E002EFED7EF2ED1
:10064000FAD70001120093968A96020E0301E16F19
:10065000FA0EE26F0001E0DF0301E12FF9D7938684
:10066000020EE16FFA0EE26F0001D6DF0301E12F07
:10067000F9D79386000112000301E26BE2510708EB
:100680001BE393968A96030E006E002EFED700D0D1
:10069000D890E13302E28A9601D08A8693967C0E46
:1006A000006E002EFED700D09386030E006E002E43
:1006B000FED700D0E22BE2D700011200030EEA6E53
:1006C000E10EE96EEF500EE0080E016E006A002E9A
:1006D000FED7012EFBD7190E006E002EFED700D0DC
:1006E000EF2EF2D712000301E16BE15107081BE383
:1006F00093968A96030E006E002EFED700D0938646
:10070000100E006E002EFED70000938681B602D038
:10071000D89001D0D880E233F90E006E002EFED7BB
:1007200000D0E12BE2D7E2C301F0000112008E0EEF
:10073000006EE2C301F0E1C302F0036A01AE05D02E
:10074000011E021E022A01E1012A015209E102C032
:1007500001F0026A080E005E015202E1006A0ED04A
:10076000D89001BE04D0023601360006F9D7030145
:10077000E2AF02D0000102D0019E0001120003018D
:10078000E551D8B4A5D0F16FE951D8B4A1D0F15F4B
:1007900005E37F0EF127D8B09BD006D0810EF15F24
:1007A000D8A096D0D8B494D0F1C300F0016A026A00
:1007B000036AF06BE6C3EFF3EF8FE7C3EEF3E8C332
:1007C000EDF3190EF16FEC51ED5F0DE2010EEE5FEE
:1007D0000AE2EF5F08E2F05F06E2F02BEF2BEE2B70
:1007E000EC51ED2728D0EB51EE5F12E2010EEF5FE6
:1007F0000FE2F05F0DE2F02BEF2BEB51EE27EC5107
:10080000ED2719E3EE2B17E1EF2B15E1F02B13D0B9
:10081000EA518009EF5F0EE2010EF05F0BE2F02B70
:10082000EA518009EF27EB51EE27E9E3EF2BE7E1EF
:10083000F02BE5D70380F12F01D00BD0D890ED3706
:10084000EE37EF37F037D890033602360136F237FD
:10085000BAD7F2A106D0D890013202320332F23375
:1008600002D0000635E0F2BF1ED0D890ED37EE374B
:10087000EF37F037EC51ED5F07E2010EEE5F04E277
:10088000EF5F02E2F05F1AE3EB51EE5F05E2010E6B
:10089000EF5F02E2F05F12E3EA518009EF5F03E2EB
:1008A000010EF05F0BE3032A09E1022A07E1012AA6
:1008B00005E1002A0DE0013202320332E6C3F1F312
:1008C000EA51F11BF1AF02D0018E06D0019E04D097
:1008D000006A016A026A036A000112000301D86B10
:1008E0000001B1DECC0E0301E16F0001C5DE440E54
:1008F0000301E16F0001C0DEC80E0301E16F0001DA
:10090000DDDE0301D85306E10001EDDE01C0D8F3BE
:10091000F8D70301000197DECC0E0301E16F00015F
:10092000ABDEBE0E0301E16F0001A6DEDCDE01C01E
:10093000D9F3D9DE01C0DAF3D6DE01C0CAF2D3DEC4
:1009400001C0CBF2D0DE01C0CCF2DAC3DCF3D9C3F4
:10095000DBF3DCC3E2F3DBC3E1F3E9DE03C0E4F382
:1009600002C0E3F301C0E2F300C0E1F303C0E8F327
:1009700002C0E7F301C0E6F300C0E5F30301EC6B4E
:10098000EB6BEA6B830EE96F0001F9DE03C0E0F365
:1009900002C0DFF301C0DEF300C0DDF3C80E0301C7
:1009A000E16F00018BDEDDC300F0DEC301F0DFC3C9
:1009B00002F0E0C303F012008E0E006ED9C301F006
:1009C000D8C302F0036A015209E102C001F0026AD1
:1009D000080E005E015202E1006A08D0D89001BE04
:1009E00004D0023601360006F9D7019E51EF05F01A
:1009F000D9C3E0F30301DD51E01BE0AF05D0D8948B
:100A0000D890D9BFD8802FD0D9C3E0F3DCC3E1F3AD
:100A1000D851E15F06E0E0AF26D0D850010AD86E89
:100A200022D0DDC3E1F3D951E15F06E0E0AF1BD096
:100A3000D850010AD86E17D0DEC3E1F3DA51E15F76
:100A400006E0E0AF10D0D850010AD86E0CD0DFC35A
:100A5000E1F3DB51E15F06E0E0AF05D0D850010AD9
:100A6000D86E01D0D890000162EF05F037DF03C0E7
:100A7000FBF202C0FAF201C0F9F200C0F8F2F2CFC4
:100A8000D8F3F29E030EA96EA69CA69EA680A8503F
:100A90000301D8BFF28ED76FD96BD7C3D8F300014B
:100AA0008BD7FBC2DBF3FAC2DAF3F9C2D9F3F8C28F
:100AB000D8F303C0DFF302C0DEF301C0DDF300C0F2
:100AC000DCF396D703E39292898202D092928992C4
:100AD00081A805D0010E0201FC6F03D000010201C4
:100AE000FC6BD76A830ED66E9E90000136EF00F045
:100AF0001E6A010E1F6E020E206E030E216E040E82
:100B0000226E050E236E82EF3CF0C00E1A6EA80E08
:100B10001B6E1C6AF2CF1BF3F29EA96AA69CA69ECE
:100B2000A680A85003011BBFF28EFF080CE0F2CF95
:100B30001BF3F29EA96AA69CA69EA680A8501BBF86
:100B4000F28E1D6E17D0060E1D6EF250006EF29ED4
:100B5000A96A1DC0A8FFA69CA69EA6840F01550EDB
:100B6000A76EAA0EA76EA682A6B2FED7A6940050C4
:100B7000F2120301C00E286EA80E296E2A6AF2CF67
:100B80001BF3F29E010EA96EA69CA69EA680A850FD
:100B90001BBFF28EFF080DE0F2CF1BF3F29E010E99
:100BA000A96EA69CA69EA680A8501BBFF28E2B6E97
:100BB00018D0030E2B6EF250006EF29E010EA96E3D
:100BC0002BC0A8FFA69CA69EA6840F01550EA76E5B
:100BD000AA0EA76EA682A6B2FED7A6940050F21265
:100BE0000301246825682668276A000184EF3CF029
:100BF000830ED56E670ED76E690ED66EF28AC00E62
:100C0000F2127DEF0AF0860E956E949C8B9C948E6A
:100C100094908B8094928B8292EF07F00301D56BB6
:100C2000D551070814E3D890D43702E28B9401D051
:100C30008B849494949C8B8C948E82BE02D0D8909A
:100C400001D0D880D637949C8B9CD52BE9D7D6C3BE
:100C500001F00001120094908B90C9C3CBF3C9C37B
:100C6000D4F30001DBDF0301D46B0001D7DF01C047
:100C7000CAF394908B800301CAC301F000011200F3
:100C800094908B900301D4690001C8DF94908B800D
:100C9000A7EF07F094908B900301CF514009D16FDB
:100CA000D46F0001BBDFD0C3D4F3B8DF94908B8046
:100CB000120094908B900301CE51A009D06FD46F95
:100CC0000001ACDFCFC3D4F3A9DF94908B80120076
:100CD00094908B900301D1518009D36FD46F0001A0
:100CE0009DDFD2C3D4F39ADF94908B8012001F0E45
:100CF0000301CE6F030ECF6F0001DBDF030E030194
:100D0000CF6FCC0ECE6F010ECE25E96E000ECF2137
:100D1000EA6EEFCFD0F31F0ED16FD0C3D2F3000134
:100D2000D7DF120094908B9023C325F323C3D4F311
:100D3000000174DF0301D46B000170DF0301D46B89
:100D400000016CDF01C024F394908B80030124C365
:100D500001F000011200020E0301CD6F140ECC6FE2
:100D60000001C5DF140E0301CF6F20C3D0F30001D3
:100D700091DF030E0301246F210E236FE96E24C35C
:100D8000EAFFEFCF25F3160ECF6F25C3D0F3000196
:100D900081DF030E0301246F210E236F010E232533
:100DA000E96E000E2421EA6EEFCF25F3170ECF6F08
:100DB00025C3D0F300016EDF030E0301CD6F0A0ED1
:100DC000CC6F000194DF0A0E0301236F0001AADF3C
:100DD00001C023F3000E030101B0010E000AD8B4D4
:100DE00002D00001F0D700011200020E0301CD6F06
:100DF000140ECC6F00017BDF140E0301CF6F20C3F4
:100E0000D0F3000147DF120E0301CF6F010ED06F48
:100E1000000140DF030E0301CD6F0A0ECC6F00010D
:100E200066DF0A0E0301236F00017CDF01C023F39C
:100E3000000E030101B0010E000AD8B402D0000177
:100E4000F0D7020ECD6F140ECC6F000150DF120EE2
:100E50000301CF6FD06B00011DDF180E0301236F5C
:100E6000000160DF01C021F3190E0301236F0001AF
:100E700059DF01C022F3030121C301F022C302F0B4
:100E800000014EEF07F01F0E0301CE6F0C0ECF6F67
:100E900000010FDF0301206B0001A7D702C01FF381
:100EA00001C01EF303011C51020804E11C6B1FB1B9
:100EB0001C2B0BD01F911CB11F81206B1FC322F371
:100EC0001EC321F3000147DF0301020ECD6FCC6F7B
:100ED00000010DDF020E0301236F000123DF01C0BB
:100EE0001DF303011D911CB11D81020ECF6F1DC3A7
:100EF000D0F30001CFDE03011C5302E0150E01D038
:100F0000120E206F040ECF6F20C3D0F30001C2DE9B
:100F10001F0E0301D16F040ED26F0001D9DE76EFF0
:100F200008F071D61D0E0301C96F000194DE01C0E7
:100F30001BF303011BA702D00001F4D71B51FF0ACA
:100F4000010BD8B402D00001EDD7000199D6196A7F
:100F5000F2BE198EF29E010E0301E16F00015EECFC
:100F600003F019BEF28E516A5A80576A566A080E0B
:100F70000301CF6FD06B00018DDE090E0301CF6F2F
:100F8000D06B000187DE0C0E0301CF6FF70ED06F20
:100F9000000180DE0D0E0301CF6F1B0ED06F00012C
:100FA00079DE0A0E0301CF6FF70ED06F000172DEFB
:100FB0000B0E0301CF6F1B0ED06F00016BDE040E12
:100FC0000301CF6FF80ED06F000164DE050E030140
:100FD000CF6F1B0ED06F00015DDE020E0301CD6FDF
:100FE000CC6B000184DE0301CF6B0D0ED06F0001CE
:100FF00051DE020E0301CF6F320ED06F00014ADEC8
:10100000030E0301CF6F400ED06F000143DE090EC7
:101010000301CF6F3F0ED06F00013CDE060E0301CF
:10102000CF6F120ED06F000135DE070E0301CF6FB8
:101030000C0ED06F00012EDE0A0E0301CF6FEE0EF4
:10104000D06F000127DE0B0E0301CF6F050ED06FAE
:10105000000120DE030E0301CD6F040ECC6F0001F2
:1010600046DE040E0301CF6F1EC0D0F3000112DE76
:10107000050E0301CF6F1FC0D0F300010BDE020E7F
:101080000301CF6F20C0D0F3000104DE030E030183
:10109000CF6F21C0D0F30001FDDD0301CF6B22C073
:1010A000D0F30001F7DD010E0301CF6F23C0D0F3B1
:1010B0000001F0DD120E0301C96F0001CCDD01C09B
:1010C0005BF0100E0301206F010E226F216B0001F7
:1010D00042DE140E0301206F040E226F720E216F88
:1010E000000139DE03011C6B0001CDD61F0E030188
:1010F000D16F040ED26F0001EBDD7EEF0AF05A9241
:1011000001011769186919691A691B691C69206B43
:101110001F6B1E6B1D6B00017FEF0AF021C350F0A7
:1011200020C34FF01FC34EF01EC34DF0ABEF09F0CC
:101130000301266B276B010E286FDA6AD96A030E4A
:101140002B6F1E0E2A6F030EEA6E220EE96E2BC362
:10115000E2FF2AC3E1FF28C329F3D890E550EE024D
:10116000F3502623F4502723292FF7D726C3DEFF79
:1011700027C326F3276BD8B0272B2A2BD8B42B2BC9
:10118000282B28510508DFE10001FEEF08F0016A75
:10119000026A006A036A0301245102E1235118E044
:1011A000100E256FD8902137223700360336245190
:1011B000035C02E12351005C07E32351005ED8A0E9
:1011C00003062451035ED88001360236252FEAD764
:1011D00000011EEF09F050C021F34FC020F34EC0B4
:1011E0001FF34DC01EF3410E0301256FC60E246F81
:1011F0004E0E236F6D0E226F00019AD7390E030138
:1012000000244D6E300E01204E6E000E02204F6EF7
:10121000000E0320506E4FC000F050C001F0026A73
:10122000036A50C020F34FC01FF350C022F34FC0D9
:1012300021F37F0E246F23690001A9D700C001F0BC
:1012400003C002F0ACEF09F003011B6B1B51040853
:1012500068E31B51240DF350036A610F016E000E09
:10126000032201C01CF303C01DF31CC3E9FF1DC30F
:10127000EAFF0A0EEF6E230E1C25E96E000E1D21FB
:10128000EA6EEF90230E1C25E96E000E1D21EA6E1A
:10129000EF82230E1C25E96E000E1D21EA6EEF84FD
:1012A000230E1C25E96E000E1D21EA6EEF98230E19
:1012B0001C25E96E000E1D21EA6EEF960F0E1C250F
:1012C000E96E000E1D21EA6EEF3C01D015D00F0E25
:1012D0001C25E96E000E1D21EA6EEFCF1EF31EC322
:1012E0006EF3000102EC00F00F0E03011C25E96E05
:1012F000000E1D21EA6EEF68210E1C25E96E000E1E
:101300001D21EA6EEC6AED521E0EEF6E100E1C25CA
:10131000E96E000E1D21EA6EEC6AED52EF6A1B2B9E
:1013200095D7D65001011527D7501623CE50152733
:10133000CF501623CC501527000E1623B250152778
:10134000B35016230301216B206B16C11FF315C187
:101350001EF30001E3D63FD702C060F001C05FF08A
:10136000040E6027605112080AE2FF0A03E15F5091
:10137000870805E2880E5F5E130E605BF3D760514D
:10138000030802E3040E602780EF0AF00301206BDC
:101390002051040873E32051240DF350036A610FB8
:1013A000016E000E032201C021F303C022F321C30A
:1013B000E9FF22C3EAFFEF500A085EE121C3E9FF1B
:1013C00022C3EAFFEF6A0B0E2125E96E000E2221EF
:1013D000EA6E1FC3ECFFED521EC3EFFF0D0E212579
:1013E000E96E000E2221EA6EEC6AED52EF6A070EFA
:1013F0002125E96E000E2221EA6EEE52EE52EC6AD1
:10140000ED52EF6AED52EF6AED52EF6A230E21259D
:10141000E96E000E2221EA6EEF80230E2125E96E8F
:10142000000E2221EA6EEF960F0E2125E96E000EC6
:101430002221EA6EEF3C01D015D00F0E2125E96E76
:10144000000E2221EA6EEFCF23F323C36EF30001D7
:1014500002EC00F00F0E03012125E96E000E22219F
:10146000EA6EEF68230E2125E96E000E2221EA6E56
:10147000EF8220C301F004D0202B8AD7FE0E016E2C
:10148000000156EF0AF003011B6B1B532EE1036AA8
:101490001B51210F016E010E032201C01CF303C07A
:1014A0001DF31F6B500E1E6F000170D71DC3EAFFA6
:1014B0001CC3E9FF01C0EFFF036A03011B51210FA9
:1014C000E96E010E0320EA6EEF50FE080CE0D890A2
:1014D0001B35036A220FE96E010E0320EA6E010E2E
:1014E000EC6EED52EF6E1B2BD0D7000181EF0AF0AE
:1014F0000201796B0001F8EF05F013D500D6A4D6F0
:10150000C2D786EF3CF05AA001D032D05A80010EEB
:10151000565C03016D6F000E57586E6F6E511A08BE
:1015200009E2FF0A03E16D51F70804E21B0E6E6F3A
:10153000F70E6D6F1E0ED16F400ED26F000168EC7A
:1015400006F00301CD6B0C0ECC6F000177EC06F0BA
:101550000C0E0301CF6F6DC3D0F300014AEC06F00F
:101560000D0E0301CF6F6EC3D0F300014AEC06F0FD
:1015700012000301BD6BBC6B94908B903A0ED46F3C
:1015800000010EEC06F00301BD51BB5D1CE303E15D
:10159000BA51BC5D18E2B9C303F0B8C3BEF3B9C316
:1015A000BFF3D46B00010EEC06F0BFC3EAFFBEC36D
:1015B000E9FF01C0EFFF0301B82BD8B4B92BBC2B56
:1015C000D8B4BD2BE1D794908B80BCC301F0BDC3D0
:1015D00002F000011200CAC3CBF3C9C3CCF303016C
:1015E000CBC301F0CCC302F000011200010E0301D5
:1015F000CD6F190ECC6F000177EC06F0190E0301C8
:10160000C96F00012BEC06F001C039F30301395317
:1016100003E1000E016E86D05AB006D0000173DFE0
:10162000000E016E03017ED057C059F056C058F02D
:10163000CD6BCC6B000177EC06F00301CF6B56C08D
:10164000D0F300014AEC06F0010E0301CF6F57C042
:10165000D0F300014AEC06F0030E03013A6F250EA9
:10166000396F3AC3B9F3B86FBB6B140EBA6F000190
:1016700080DF38C3CAF337C3C9F3ADDF02C038F324
:1016800001C037F3030126511A0805E2FF0A19E1E8
:101690002551F70816E3030E3A6F250EE96E3AC39B
:1016A000EAFFEFB00ED02ABF0CD029B90AD02851DA
:1016B000040805E2FF0A05E12751EE0802E329BF0D
:1016C00001D0FF0026C357F025C356F022C303F014
:1016D00021C339F322C33AF322C3EAFF21C3E9FF4E
:1016E000030EE26E310EE16E060E016EE6CFEEFFE6
:1016F000012EFCD724C303F023C3E9FF03C0EAFF94
:10170000EF68385108080BE1375303E037510608FA
:1017100006E123C3E9FF24C3EAFF37C3EFFF5A9072
:10172000010E016E000100EF3BF003014CC301F01C
:101730004DC303F04CC34EF34DC34FF34CC3E9FF0D
:101740004DC3EAFFECCF51F3ED52EFCF50F351C34D
:10175000CAF350C3C9F300013EDF4FC3EAFF4EC3D3
:10176000E9FF02C0ECFFED5201C0EFFF020E0301E2
:101770004C25016E000E4D21036E01C04EF34F6FDC
:10178000020E4C25E96E000E4D21EA6EECCF51F3AE
:10179000ED52EFCF50F351C3CAF350C3C9F3000168
:1017A0001ADF4FC3EAFF4EC3E9FF02C0ECFFED5260
:1017B00001C0EFFF060E03014C25016E000E4D2106
:1017C000036E01C04EF34F6F060E4C25E96E000EFE
:1017D0004D21EA6EECCF51F3ED52EFCF50F351C3F0
:1017E000CAF350C3C9F30001F6DE4FC3EAFF4EC38C
:1017F000E9FF02C0ECFFED5201C0EFFF1200030E43
:101800000301B96F300EB86FBB6B1C0EBA6F0001CD
:10181000B0DE79DE030E03014D6F300E4C6F000118
:1018200084DF0301302D08D0315306E1345106081E
:1018300003E13551040803E0000E016E51D036512A
:1018400002080AE1375308E12FC303F02EC3E9FF72
:101850002FC3EAFFEF6A16D0362D0BD0375309E1BC
:101860002FC303F02EC3E9FF2FC3EAFF010EEF6E73
:1018700009D02EC3E9FF2FC3EAFF020EEF6E000E60
:10188000016E2ED01A50485D29E11B50495D26E1BA
:101890001C504A5D23E11D504B5D20E12CC3E9FF44
:1018A0002DC3EAFF030EE26E380EE16E060E016EE6
:1018B000E6CFEEFF012EFCD7060E2C25E96E000EBA
:1018C0002D21EA6E3EC3EFFF3FC3ECFF40C3ECFFA8
:1018D00041C3ECFF010E016E03D002D0000E016E79
:1018E000000165EF0FF01F0E0301C96F00012BEC23
:1018F00006F001C0ABF3000E030101B6010E000AB1
:1019000002E1000E01D0FF0E016E00011200C3C300
:1019100051F0070E0301C4271C0EC523CD6B020E28
:10192000CC6F000177EC06F0030E0301C76FC40E05
:10193000C66FE96EC7C3EAFFEFCFC8F3CF6BC8C36A
:10194000D0F300014AEC06F0030E0301C76FC40E8A
:10195000C66F010EC625E96E000EC721EA6EEFCFF5
:10196000C8F3010ECF6FC8C3D0F300014AEC06F0F4
:10197000030E0301C76FC40EC66FE96EC7C3EAFF4B
:10198000EFCFC8F3020ECF6FC8C3D0F300014AEC0B
:1019900006F0030E0301C76FC40EC66F010EC62505
:1019A000E96E000EC721EA6EEFCFC8F3030ECF6FCA
:1019B000C8C3D0F300014AEC06F0120094908B905B
:1019C0007A0E0301D46F00010EEC06F0CDC3D4F300
:1019D0000EEC06F094908B80120094908B907A0E0F
:1019E0000301D46F00010EEC06F00301D1C303F034
:1019F000D051D8B4D107D007031012E0CFC303F001
:101A0000CEC3E9FFCFC3EAFFEFCFD2F3D2C3D4F303
:101A100000010EEC06F00301CE2BD8B4CF2BE6D795
:101A200094908B80000112000301CD6B020ECC6FED
:101A3000000177EC06F0020E0301CF6FF80ED06FB5
:101A400000014AEC06F0030E0301CF6F1B0ED06FAE
:101A500000014AEC06F0060E0301CA271C0ECB2338
:101A6000030ECD6FCA0ECC6FE96ECDC3EAFFEFCF88
:101A7000CEF3060ECF6FCEC3D0F300014AEC06F0D2
:101A8000030E0301CD6FCA0ECC6F010ECC25E96E9B
:101A9000000ECD21EA6EEFCFCEF3070ECF6FCEC38F
:101AA000D0F300014AEC06F00301CD6B000186DFA4
:101AB000C8C3CFF3C7C3CEF30301D16B060ED06FFB
:101AC00000018BDF0301CD6B1E0ECC6FCDC3CFF3B6
:101AD000CE6FD16B060ED06F00017FDF080E0301C1
:101AE000CD6F00016BDF0301C95302E1000E01D08D
:101AF000060ECC6FCD6F000161DF12001C0E0301DA
:101B0000C96F00012BEC06F001C0B6F3000E030113
:101B100001B2010E000A10E01F0ED16F800ED26FCD
:101B2000000168EC06F01F0E0301CE6F800ECF6F30
:101B3000000159EC06F003011C0ECE6F0A0ECF6FA8
:101B4000000159EC06F01F0E0301D16F080ED26F91
:101B5000000168EC06F05B500508D8A4E2D01C0E2A
:101B60000301C96F00012BEC06F001C0B6F30301BD
:101B700001500A0BD8A402D00001F1D71C0EC96F86
:101B800000012BEC06F001C0B6F3000E030101B218
:101B9000010E000AD8B4C6D01F0ECE6F080ECF6F4C
:101BA000000159EC06F00301CD6BCC6B000177EC22
:101BB00006F00301C96B00012BEC06F001C0AAF38B
:101BC000010E0301C96F00012BEC06F001C0ABF35D
:101BD000060E0301C96F00012BEC06F001C0ACF347
:101BE000070E0301C96F00012BEC06F001C0ADF335
:101BF0000301AC2BD8B4AD2BCF6BACC3D0F3000139
:101C00004AEC06F0010E0301CF6FADC3D0F3000123
:101C10004AEC06F0030E0301B76FAE0EB66FB7C302
:101C2000B9F3B86FBB6B070EBA6F0001A2DC0301FA
:101C3000B56BB5510F0867E31C0EC96F00012BECA3
:101C400006F001C0B6F3000E030101B2010E000A56
:101C500055E0B1AB53D01F0ED16F800ED26F000193
:101C600068EC06F01F0E0301CE6F800ECF6F0001EF
:101C700059EC06F01C0E0301CE6F0A0ECF6F000167
:101C800059EC06F01F0E0301D16F080ED26F000150
:101C900068EC06F01C0E0301C96F00012BEC06F086
:101CA00001C0B6F3030101500A0BD8A402D0000111
:101CB000F1D71F0ECE6F080ECF6F000159EC06F062
:101CC0000301CF6BACC3D0F300014AEC06F0010E68
:101CD0000301CF6FADC3D0F300014AEC06F0030E51
:101CE0000301B76FAE0EB66FB7C3B9F3B86FBB6B76
:101CF000070EBA6F00013DDC03D0030104D00001E0
:101D00000301B52B96D7CF6BAAC3D0F300014AECE1
:101D100006F0010E0301CF6FABC3D0F300014AEC14
:101D200006F0030100011200010E0301AA6F000179
:101D3000DADD01C04BF303014B3D03D0000E016E11
:101D4000B0D04BC3C3F3C56BC46B0001E0DD03012E
:101D5000306B010E2F6F080E326F316B060E336F32
:101D6000040E346F2E2D0AD0366B010E356F41698B
:101D70004269436944694569466911D0366B020E70
:101D8000356F2CC3E1FF2DC3E2FF030EEA6E410E57
:101D9000E96E060E016EE6CFEEFF012EFCD7030EB4
:101DA000EA6E370EE96EE26A1E0EE16E060E016EF5
:101DB000E6CFEEFF012EFCD71DC040F31CC03FF361
:101DC0001BC03EF31AC03DF3060E2C25E96E000E33
:101DD0002D21EA6EEFCF00F0ECCF01F0ECCF02F056
:101DE000ECCF03F000503D194C6F01503E194D6F80
:101DF00002503F194E6F035040194F6F4C5124143D
:101E0000006E4D512514016E4E512614026E4F5135
:101E10002714036E005206E1015204E1025202E16E
:101E2000035209E02BC04AF32AC049F329C048F302
:101E300028C047F316D0060E2C25E96E000E2D2182
:101E4000EA6EEFCF00F0ECCF01F0ECCF02F0ECCF78
:101E500003F000C047F301C048F302C049F303C0D8
:101E60004AF3030E4D6F2F0E4C6F00015EDC030E24
:101E70000301C86F410EC76F060EC96FCB6B1C0EF6
:101E8000CA6F0001D1DD030E0301CF6F2F0ECE6F9D
:101E9000D16B1C0ED06F0001A0DD30DE010E016E93
:101EA0000301000191EF0FF0000E5AB2010E000A7B
:101EB00001E02FD0030E03012D6F210E2C6F030EB6
:101EC0002F6F2B0E2E6F00019AD4015201E130D0FA
:101ED00083EC0AF003012B531AE1010EEA6E170E90
:101EE000E96E030EE26E210EE16E060E016EE6CF84
:101EF000EEFF012EFCD72AC320F129C31FF128C30E
:101F00001EF127C31DF1000113D003D003015A8233
:101F10000001030E03012D6F210E2C6F2E6B0001AB
:101F200003D7015202E05A9203D0000E016E02D094
:101F3000010E016E1DEF3BF0140E58240301806F5B
:101F4000000E5920816F7A5180257E6F7B5181214F
:101F50007F6F7F511A0809E2FF0A03E17E51F708FB
:101F600004E2F80E7E5F1B0E7F5BCD6B100ECC6F14
:101F7000000177EC06F0100E0301CF6F7EC3D0F3A3
:101F800000014AEC06F0110E0301CF6F7FC3D0F3BE
:101F900000014AEC06F0010E03017C5D006E000EAC
:101FA0007D59036E00507E2703507F237F511A080E
:101FB00009E2FF0A03E17E51F70804E2F80E7E5FB2
:101FC0001B0E7F5B120ECF6F7EC3D0F300014AEC75
:101FD00006F0130E0301CF6F7FC3D0F300014AEC6C
:101FE00006F01F0E0301D16F300ED26F000168ECB6
:101FF00006F01F0E0301C96F00012BEC06F001C0B3
:1020000080F3000E030101BA010E000AD8B402D019
:102010000001EFD7160EC96F00012BEC06F001C0CE
:102020007FF3170E0301C96F00012BEC06F001C00E
:102030007EF303017EC301F07FC302F000011200B2
:10204000140E58240301566F000E5920576F525139
:102050005625546F53515721556F55511A0809E2AF
:10206000FF0A03E15451F70804E2F80E545F1B0E17
:10207000555BCD6BCC6B000177EC06F00301CF6BA9
:1020800054C3D0F300014AEC06F0010E0301CF6FF8
:1020900055C3D0F300014AEC06F0020E0301CF6FE6
:1020A00054C3D0F300014AEC06F0030E0301CF6FD6
:1020B00055C3D0F300014AEC06F01200020E0301F2
:1020C000C325016E000EC421036E01C0C5F3C66FA7
:1020D000020EC325E96E000EC421EA6EECCFC8F3F0
:1020E000ED52EFCFC7F3C8C3CAF3C7C3C9F30001AA
:1020F000EBEC0AF0C6C3EAFFC5C3E9FF02C0ECFF80
:10210000ED5201C0EFFF040E0301C325016E000E66
:10211000C421036E01C0C5F3C66F040EC325E96E6A
:10212000000EC421EA6EECCFC8F3ED52EFCFC7F337
:10213000C8C3CAF3C7C3C9F30001EBEC0AF0C6C3B6
:10214000EAFFC5C3E9FF02C0ECFFED5201C0EFFF9B
:102150000A0E0301C325016E000EC421036E01C0E7
:10216000C5F3C66F0A0EC325E96E000EC421EA6EE0
:10217000ECCFC8F3ED52EFCFC7F3C8C3CAF3C7C360
:10218000C9F30001EBEC0AF0C6C3EAFFC5C3E9FFDF
:1021900002C0ECFFED5201C0EFFF1200030E03017D
:1021A000406F2B0E3F6F40C3B9F3B86FBB6B140E7B
:1021B000BA6F0001B9EC0AF003012B51F00B400893
:1021C00003E0000E016E58D02B510F0B006E00344F
:1021D0005E6E5E36FC0E5E167B6B7A6B7D6B5EC050
:1021E0007CF30001A9DE02C02AF301C029F3030138
:1021F000536B5EC052F3000123DF030129512A1102
:1022000003E0000E016E38D0030EC46F2B0EC36FB7
:10221000000154DF0301215122110CE021C3E9FF29
:1022200022C3EAFF3BC3EFFF3CC3ECFF3DC3ECFF1F
:102230003EC3ECFF060E2325E96E000E2421EA6E54
:1022400037C3EFFF38C3ECFF39C3ECFF3AC3ECFFF1
:1022500025C3E9FF26C3EAFF34C3EFFF27C3E9FF25
:1022600028C3EAFF5E502D5D006E000E2E5900C09F
:10227000EFFFEC6E010E016E000138EF3BF0030141
:10228000BB6BBA6BB96BB86BD890AF31B16FAE3175
:10229000B06FADC3B3F3ACC3B2F3B1C303F0B0518D
:1022A000D8B4B107B007031017E0B3C303F0B2C34B
:1022B00000F0020EB227D8B0B32B00C0E9FF03C074
:1022C000EAFFECCF03F0ED52EF50B8270350B923EB
:1022D000000EBA23BB23E1D7AE51010B006E036A97
:1022E000005003100AE0B2C3E9FFB3C3EAFFEF50A6
:1022F000B827000EB923BA23BB23BBC3B7F3BAC3B5
:10230000B6F3B9C3B5F3B8C3B4F3B7C3B1F3B6C347
:10231000B0F3B05302E1B1531FE0BB6BBA6BBF6BBC
:10232000BE6BB9C3BDF3B8C3BCF3026A036AB05154
:10233000B825B86FB151B921B96F0250BE21BA6F3B
:102340000350BF21BB6FBBC3B7F3BAC3B6F3B9C366
:10235000B5F3B8C3B4F3D9D7B9C303F0031EB8516A
:10236000FF0A016E03C002F00001120094908B90EE
:102370003A0E0301D46F00010EEC06F00301D46B9A
:1023800000010EEC06F001C0AEF394908B800301C7
:10239000AEC301F0000112000301AA5307E1AB53E1
:1023A00005E1FF0E016E026EA1D017D0AA2D15D047
:1023B000AB5313E10001DADF0301AF6B01C0AEF3F1
:1023C00001C003F0000E006A0006001AFF0E031A97
:1023D00000C001F003C002F089D0CD6BCC6B0001CE
:1023E00077EC06F00301C96B00012BEC06F001C08D
:1023F000ACF3010E0301C96F00012BEC06F001C024
:10240000ADF3100E0301CF6FACC3D0F300014AEC63
:1024100006F0110E0301CF6FADC3D0F300014AECFB
:1024200006F00301AD511B081BE303E1AC51F708B3
:1024300017E3010EAA5D006E000EAB59036E00504B
:10244000AC270350AD23AD511A0809E2FF0A03E19E
:10245000AC51F70804E2F80EAC5F1B0EAD5B0AD07E
:10246000010EAA5D006E000EAB59036E0050AC2742
:102470000350AD23120ECF6FACC3D0F300014AEC72
:1024800006F0130E0301CF6FADC3D0F300014AEC89
:1024900006F01F0E0301D16F300ED26F000168EC01
:1024A00006F01F0E0301C96F00012BEC06F001C0FE
:1024B000AEF3000E030101BA010E000AD8B402D037
:1024C0000001EFD7160EC96F00012BEC06F001C01A
:1024D000ACF3170E0301C96F00012BEC06F001C02D
:1024E000ADF30301ACC301F0ADC302F00001120073
:1024F0005E5003014E25506F000E4F21516F536FF8
:1025000050C352F300019CDD1200B5C3B6F3B4C34F
:10251000B7F3B3C3B8F3B2C3B9F3B6C300F0B7C3EC
:1025200001F0B8C302F0B9C303F012000301AAC35B
:1025300001F0ABC303F0AAC3ACF3ABC3ADF3AAC3C2
:10254000E9FFABC3EAFFECCFAFF3ED52EFCFAEF351
:10255000AFC3CAF3AEC3C9F30001EBEC0AF0ADC3DD
:10256000EAFFACC3E9FF02C0ECFFED5201C0EFFF90
:10257000020E0301AA25016E000EAB21036E01C0FD
:10258000ACF3AD6F020EAA25E96E000EAB21EA6E28
:10259000ECCFAFF3ED52EFCFAEF3AFC3CAF3AEC3A0
:1025A000C9F30001EBEC0AF0ADC3EAFFACC3E9FFED
:1025B00002C0ECFFED5201C0EFFF040E0301AA259B
:1025C000016E000EAB21036E01C0ACF3AD6F040EC3
:1025D000AA25E96E000EAB21EA6EEFCFAEF3ECCF89
:1025E000AFF3ECCFB0F3ECCFB1F3B1C3B5F3B0C3FD
:1025F000B4F3AFC3B3F3AEC3B2F3000186DFADC330
:10260000EAFFACC3E9FF00C0EFFF01C0ECFF02C06E
:10261000ECFF03C0ECFF080E0301AA25016E000EBB
:10262000AB21036E01C0ACF3AD6F080EAA25E96EB5
:10263000000EAB21EA6EEFCFAEF3ECCFAFF3ECCFF1
:10264000B0F3ECCFB1F3B1C3B5F3B0C3B4F3AFC3E0
:10265000B3F3AEC3B2F3000158DFADC3EAFFACC3BE
:10266000E9FF00C0EFFF01C0ECFF02C0ECFF03C0B8
:10267000ECFF0E0E0301AA25016E000EAB21036EC6
:1026800001C0ACF3AD6F0E0EAA25E96E000EAB21B2
:10269000EA6EECCFAFF3ED52EFCFAEF3AFC3CAF3B8
:1026A000AEC3C9F30001EBEC0AF0ADC3EAFFACC363
:1026B000E9FF02C0ECFFED5201C0EFFF100E030175
:1026C000AA25016E000EAB21036E01C0ACF3AD6F05
:1026D000100EAA25E96E000EAB21EA6EECCFAFF327
:1026E000ED52EFCFAEF3AFC3CAF3AEC3C9F30001EF
:1026F000EBEC0AF0ADC3EAFFACC3E9FF02C0ECFFAC
:10270000ED5201C0EFFF120E0301AA25016E000E6B
:10271000AB21036E01C0ACF3AD6F120EAA25E96EBA
:10272000000EAB21EA6EECCFAFF3ED52EFCFAEF37C
:10273000AFC3CAF3AEC3C9F30001EBEC0AF0ADC3FB
:10274000EAFFACC3E9FF02C0ECFFED5201C0EFFFAE
:102750001200FE0E0301546F536B53510408D8A0AE
:102760007AD05351240DF350036A610F016E000EAD
:10277000032201C051F303C052F351C3E9FF52C316
:10278000EAFFEF500A0865E00B0E5125E96E000ED6
:102790005221EA6EECCF56F3ED52EFCF55F3020E15
:1027A0004D25E96E000E4E21EA6EECCF03F0ED529E
:1027B000EF50555D4EE10350565D4BE151C3E9FFCB
:1027C00052C3EAFFEF5202E153C354F30D0E5125F9
:1027D000E96E000E5221EA6EECCF56F3ED52EFCFC8
:1027E00055F34DC3E9FF4EC3EAFFECCF03F0ED52C2
:1027F000EF50555D2EE10350565D2BE1070E51253C
:10280000E96E000E5221EA6EEFCF55F3ECCF56F38E
:10281000ECCF57F3ECCF58F3060E4F25E96E000EC0
:102820005021EA6EEFCF00F0ECCF01F0ECCF02F0D8
:10283000ECCF03F00050555D0CE10150565D09E10D
:102840000250575D06E10350585D03E153C301F0A8
:102850006ED0532B82D75451FE0803E1FE0E016E59
:1028600066D05451240DF350036A610F016E000EBF
:10287000032201C051F303C052F3010E5125016E32
:10288000000E5221036E01C055F3566FEA6E01C06F
:10289000E9FF50C3E2FF4FC3E1FF0A0E016EE6CF2E
:1028A000EEFF012EFCD70D0E5125016E000E5221B8
:1028B0004DC3E9FF4EC3EAFFECCF03F0ED52EFCF7B
:1028C00057F3EA6E01C0E9FF03C0ECFFED5257C3B6
:1028D000EFFF230E5125E96E000E5221EA6EEF96AE
:1028E0000F0E5125E96E000E5221EA6EEF3C01D029
:1028F00015D00F0E5125E96E000E5221EA6EEFCF72
:1029000055F355C36EF3000102EC00F00F0E030106
:102910005125E96E000E5221EA6EEF68230E512513
:10292000E96E000E5221EA6EEF8254C301F00001FD
:10293000ADEF1DF0F29A53C06EF352C06DF3F28A00
:1029400003016DC301F06EC302F0000112000F0E0F
:1029500003016B25E96E000E6C21EA6EEF3C01D09D
:102960001CD00F0E6B25E96E000E6C21EA6EEFCFC6
:102970006DF36DC36EF3000102EC00F00F0E030166
:102980006B25E96E000E6C21EA6EEF68230E6B2555
:10299000E96E000E6C21EA6EEF82070E6B25E96E80
:1029A000000E6C21EA6EEE52EE52EC6AED52EF6AC6
:1029B000ED52EF6AED52EF6A0D0E6B25E96E000ED7
:1029C0006C21EA6EEC6AED52EF6A230E6B25E96E1C
:1029D000000E6C21EA6EEFA604D0000183EC0AF031
:1029E0000301230E6B25E96E000E6C21EA6EEF9653
:1029F000210E6B25E96E000E6C21EA6EEC6AED5239
:102A00001E0EEF6E230E6B25E96E000E6C21EA6E32
:102A1000EF98230E6B25E96E000E6C21EA6EEFA095
:102A200006D06BC3E9FF6CC3EAFFEF6A06D06BC345
:102A3000E9FF6CC3EAFF0A0EEF6E100E6B25E96E1C
:102A4000000E6C21EA6EEC6AED52EF6A0001120092
:102A50001F0E0301C96F00012BEC06F001C0ABF3A0
:102A6000000E030101B6010E000A02E0000E01D0C3
:102A7000010E016E00011200010E0301CD6F190E4F
:102A8000CC6F000177EC06F0190E0301C96F00014D
:102A90002BEC06F001C0AAF30301CD6B0E0ECC6F38
:102AA000000177EC06F00E0E0301C96F00012BEC5C
:102AB00006F001C0ACF30F0E0301C96F00012BEC4F
:102AC00006F001C0ADF3010E0301CD6F190ECC6FFE
:102AD000000177EC06F0190E0301C96F00012BEC21
:102AE00006F001C0AEF30301AA51015CD8B402D0D4
:102AF0000001CAD7CD6B0C0ECC6F000177EC06F04D
:102B00000C0E0301C96F00012BEC06F001C0AAF303
:102B10000D0E0301C96F00012BEC06F001C0ABF3F1
:102B20000301AB51AD5D16E303E1AC51AA5D12E2C6
:102B3000AA51AC5D006EAB51AD59036E0050FF0A57
:102B4000F80F006E1B0E035600C001F003C002F028
:102B50001CD01BD0AA51AC5D09E1AB51AD5D06E1C3
:102B6000F70E016E1B0E026E10D00FD0AC51AA5D95
:102B7000AE6FAD51AB59AF6F010EAE5D006E000E82
:102B8000AF59036E00C001F0026E000104EF17F0B0
:102B9000060E0301C325C96F1C0EC421CA6F010EA6
:102BA000C925C76F000ECA21C86FCD6B100ECC6F40
:102BB000000177EC06F0100E0301CF6FC7C3D0F30E
:102BC00000014AEC06F0110E0301CF6FC8C3D0F329
:102BD00000014AEC06F0010E0301C55D006E000E17
:102BE000C659036E0050C7270350C823120ECF6F7B
:102BF000C7C3D0F300014AEC06F0130E0301CF6FF8
:102C0000C8C3D0F300014AEC06F01F0E0301D16FD8
:102C1000300ED26F000168EC06F01F0E0301C96F81
:102C200000012BEC06F001C0C9F3000E030101BA4C
:102C3000010E000AD8B402D00001EFD7160EC96FFA
:102C400000012BEC06F001C0C8F3170E0301C96F99
:102C500000012BEC06F001C0C7F30301C7C301F06C
:102C6000C8C302F000011200140E5E6E450E03018F
:102C7000AF6FB06B140EAD25B16F000EAE21B26F09
:102C80005C2AD8B45D2A5DC0B4F35CC0B3F3B66B04
:102C9000B56B640EB76FACC3B8F3BA6BB96B1DC03C
:102CA000BEF31CC0BDF31BC0BCF31AC0BBF3060EC1
:102CB000AA25E96E000EAB21EA6EEFCFBFF3ECCF91
:102CC000C0F3ECCFC1F3ECCFC2F3030EC46FAF0E71
:102CD000C36F00015EEC10F00301AAC301F0ABC3A7
:102CE00003F0AAC3C3F3ABC3C4F3140EAD25C56F81
:102CF000000EAE21C66FABC3C8F3AAC3C7F3C96B3E
:102D0000CB6FC5C3CAF3000114EC0DF0030E030131
:102D1000C46FAF0EC36FC4C3CFF3CE6FD16B140EAD
:102D2000D06F0001EDEC0CF00301C46BC36BC66BFC
:102D3000140EC56F00012CDF02C0BAF301C0B9F355
:102D400051C0C3F30301C56B0A0EC46F000187ECC9
:102D50000CF0030E0301C46FB90EC36FC4C3CFF3ED
:102D6000CE6FD16B020ED06F0001EDEC0CF051C0B4
:102D7000C3F30301C56B140EC46F000187EC0CF0A4
:102D8000000E016E026E1200010E0301AA6F000117
:102D90005FDE0152F9E00301813D08D0010EAA6F08
:102DA000000173EC0CF001C081F30301813D01D0FF
:102DB00003D181C3C3F3C56B140EC46F000187EC4C
:102DC0000CF075C387F374C386F377C389F376C3B6
:102DD00088F37BC38DF37AC38CF379C38BF378C309
:102DE0008AF37FC391F37EC390F37DC38FF37CC3DB
:102DF0008EF33F0E03019315936FF00E9215926FB1
:102E000080C393F3000138D602C095F301C094F358
:102E10000301955303E19451280805E2280E945FBD
:102E2000000E955B02D0956B946B976B966B996BCC
:102E3000986B030EAB6F860EAA6F000196EC12F032
:102E4000140E03018227000E832380A30FD0040EEB
:102E50008227000E8323020E9A6F040E9B6F9C6FD5
:102E60009D6B0F0E92156009926F04D00F0E921594
:102E70005009926F1DC0A1F31CC0A0F31BC09FF3AB
:102E80001AC09EF3060E7225E96E000E7321EA6EDB
:102E9000EFCF00F0ECCF01F0ECCF02F0ECCF03F07D
:102EA00000C0A2F301C0A3F302C0A4F303C0A5F3C2
:102EB000A66B060EA76F83C3A9F382C3A8F3A9C3A9
:102EC000CAF3A8C3C9F30001EBEC0AF002C0A9F3EE
:102ED00001C0A8F3030E0301AB6F9E0EAA6FABC334
:102EE000ADF3AC6FAF6B0C0EAE6F00013FEC11F0A9
:102EF00001C096F30301961F02C097F3971F97C373
:102F000085F396C384F373C3ABF372C3AAF3060EBF
:102F1000AC6F83C3AEF382C3ADF30001A5DE030E35
:102F20000301AB6F860EAA6FABC3CFF3CE6FD16B2D
:102F3000140ED06F0001EDEC0CF0030180A30ED055
:102F4000030EAB6F9A0EAA6FABC3CFF3CE6FD16BEC
:102F5000040ED06F0001EDEC0CF0030181C3C3F34C
:102F6000C56B140EC46F000187EC0CF083C3ABF388
:102F700082C3AAF3CCEC11F002C085F301C084F344
:102F800081C3C3F30301C56B240EC46F000187EC3A
:102F90000CF085C3CDF3DEEC0CF084C3CDF3DEEC96
:102FA0000CF081C3C3F30301C56BC46B000187EC54
:102FB0000CF07EEC0DF003010001120003014D51F5
:102FC000240DF350036A610F016E000E032201C04D
:102FD00064F303C065F3666B1E0E6425E96E000E94
:102FE0006521EA6EEF6A1F0E6425016E000E6521F1
:102FF000036E01C06BF36C6F00019CDC6CC3EAFFD5
:103000006BC3E9FF02C0ECFFED5201C0EFFF210EE0
:1030100003016425E96E000E6521EA6EEC6AED524B
:103020001E0EEF6E0D0E5025E96E000E5121EA6E58
:10303000EFA41ED0000183EC0AF0030164C301F089
:1030400065C303F064C36BF365C36CF3230E64259F
:10305000E96E000E6521EA6EEFA002D0000E01D0ED
:10306000010E6CC3EAFF6BC3E9FFEF6EF3EF1CF0D8
:10307000160E6425E96E000E6521EA6EEFCF58F357
:10308000ECCF59F3ECCF5AF3ECCF5BF30E0E502597
:10309000E96E000E5121EA6EECCF03F0ED52EFCF56
:1030A0006BF303C06CF36D6B6E6B080E5025E96E0D
:1030B000000E5121EA6EEFCF00F0ECCF01F0ECCF23
:1030C00002F0ECCF03F00050585D006E01505959EA
:1030D000016E02505A59026E03505B59036E005044
:1030E0006B5F01506C5B02506D5B03506E5B100EAA
:1030F0006425E96E000E6521EA6EECCF03F0ED5217
:10310000EFCF00F003C001F0026A036A00506B5D6C
:10311000676F01506C59686F02506D59696F0350A9
:103120006E596A6F6AAF0AD0140E6425E96E000EFC
:103130006521EA6EEC6AED52EF6A0AD0140E64253E
:10314000E96E000E6521EA6E54C3EFFF55C3ECFF34
:1031500064C3E9FF65C3EAFFEF2CB5D00D0E50251F
:10316000E96E000E5121EA6EEFB212D0000183EC3D
:103170000AF00D0E03015025E96E000E5121EA6E92
:10318000EFA804D0040E666FB8EF1CF0F3EF1CF04C
:103190001A0E6425016E000E652101C06BF36C6F81
:1031A000040E5025E96E000E5121EA6EEFCF6DF34B
:1031B000ECCF6EF3ECCF6FF3ECCF70F352516D2781
:1031C00053516E23000E6F237023010E6D25006E88
:1031D000000E6E21016E000E6F21026E000E702136
:1031E0006CC3EAFF6BC3E9FF00C0EFFF01C0ECFF57
:1031F00002C0ECFFEC6E1A0E6425E96E000E65212C
:10320000EA6EEFCF54F3ECCF55F3ECCF56F3ECCF9F
:1032100057F30D0E5025E96E000E5121EA6EEFB8FE
:103220000DD064C3E9FF65C3EAFF020EEF6E000133
:1032300083EC0AF0120E0301666F9AD364C3E9FFB0
:1032400065C3EAFF030EEF6E100E666F140E642561
:10325000016E000E6521036E6C6F0E0E5025E96E37
:10326000000E5121EA6EECCF03F0ED52EFCF6DF37B
:103270006CC3EAFF01C0E9FF03C0ECFFED526DC370
:10328000EFFF525153111AE0230E6425E96E000E30
:103290006521EA6EEF86120E6425E96E000E652147
:1032A000EA6E53C3ECFFED5252C3EFFF230E6425C9
:1032B000E96E000E6521EA6EEF8404D0000183EC14
:1032C0000AF0030155D364C3E9FF65C3EAFFEF5277
:1032D000D8A4BFD0000183EC0AF00D0E03015025E5
:1032E000E96E000E5121EA6EEFB203D0040E666F54
:1032F0003FD31A0E6425016E000E652101C06BF3E9
:103300006C6F040E5025E96E000E5121EA6EEFCF6E
:103310006DF3ECCF6EF3ECCF6FF3ECCF70F3525153
:103320006D2753516E23000E6F237023010E6D2500
:10333000006E000E6E21016E000E6F21026E000EF7
:1033400070216CC3EAFF6BC3E9FF00C0EFFF01C04F
:10335000ECFF02C0ECFFEC6E140E6425016E000E53
:103360006521036E6C6F0E0E5025E96E000E512123
:10337000EA6EECCF03F0ED52EFCF6DF36CC3EAFFD2
:1033800001C0E9FF03C0ECFFED526DC3EFFF010E7A
:103390006425016E000E6521036E01C06BF36C6F36
:1033A000EA6E01C0E9FF4FC3E2FF4EC3E1FF0A0E20
:1033B000016EE6CFEEFF012EFCD70D0E6425016EE7
:1033C000000E652150C3E9FF51C3EAFFECCF03F0C3
:1033D000ED52EFCF6DF3EA6E01C0E9FF03C0ECFFE1
:1033E000ED526DC3EFFF64C3E9FF65C3EAFF020E50
:1033F000EF6E160E6425E96E000E6521EA6EEE5240
:10340000EE52EE52EDCF03F0EDCF02F0EDCF01F032
:10341000EFCF00F0010EEE26000EEE22EE22ED229E
:1034200003C05BF302C05AF301C059F300C058F364
:103430001A0E6425E96E000E6521EA6EEFCF54F393
:10344000ECCF55F3ECCF56F3ECCF57F3120E666F7B
:103450008FD21A0E6425E96E000E6521EA6EEFCF59
:103460005CF3ECCF5DF3ECCF5EF3ECCF5FF3160EC5
:103470006425E96E000E6521EA6EEFCF60F3ECCFB4
:1034800061F3ECCF62F3ECCF63F3040E5025E96EE9
:10349000000E5121EA6EEFCF54F3ECCF55F3ECCF91
:1034A00056F3ECCF57F3026A036A52515427535133
:1034B00055230250562303505723160E6425E96EF8
:1034C000000E6521EA6EEFCF58F3ECCF59F3ECCF45
:1034D0005AF3ECCF5BF3040E5025E96E000E512138
:1034E000EA6EEFCF6BF3ECCF6CF3ECCF6DF3ECCF78
:1034F0006EF35C516B5DD8A42DD25D516C5DD8A488
:1035000029D25E516D5DD8A425D25F516E5DD8A4DD
:1035100021D264C3E9FF65C3EAFFEF50020843E12B
:103520000D0E5025E96E000E5121EA6EEFA836D03F
:103530001A0E6425E96E000E6521EA6E54C3EFFF92
:1035400055C3ECFF56C3ECFF57C3ECFF64C3E9FF60
:1035500065C3EAFF030EEF6E525153111AE0230EBA
:103560006425E96E000E6521EA6EEF86120E642571
:10357000E96E000E6521EA6E53C3ECFFED5252C3B3
:10358000EFFF230E6425E96E000E6521EA6EEF84DD
:1035900004D0000183EC0AF0030104D0000183ECA5
:1035A0000AF00301D6D11A0E6425E96E000E6521DA
:1035B000EA6E54C3EFFF55C3ECFF56C3ECFF57C38D
:1035C000ECFF64C3E9FF65C3EAFFEF500308D8A42A
:1035D000D9D00D0E5025E96E000E5121EA6EEFA8EC
:1035E0002DD0230E6425E96E000E6521EA6EEFB240
:1035F00025D00F0E6425E96E000E6521EA6EEF3CC2
:1036000001D01CD00F0E6425E96E000E6521EA6E14
:10361000EFCF6BF36BC36EF3000102EC00F00F0E03
:1036200003016425E96E000E6521EA6EEF68230E42
:103630006425E96E000E6521EA6EEF820D0E5025BD
:10364000E96E000E5121EA6EEFA050D0110E666FA8
:10365000160E6425E96E000E6521EA6EEE52EE52FA
:10366000EE52EDCF03F0EDCF02F0EDCF01F0EFCF52
:1036700000F0010EEE26000EEE22EE22ED2203C037
:103680005BF302C05AF301C059F300C058F31A0E9D
:103690006425E96E000E6521EA6E010EEF24006ECE
:1036A000000EEC20016E000EEC20026E000EEC20ED
:1036B000ED52ED52ED5200C0EFFF01C0ECFF02C031
:1036C000ECFFEC6E1A0E6425E96E000E6521EA6EC1
:1036D000EFCF54F3ECCF55F3ECCF56F3ECCF57F3D9
:1036E00064C3E9FF65C3EAFF090EEF6E525153113F
:1036F00044E0230E6425E96E000E6521EA6EEFB604
:103700001BD0230E6425E96E000E6521EA6EEF865C
:10371000120E6425E96E000E6521EA6E53C3ECFFBC
:10372000ED5252C3EFFF230E6425E96E000E6521B2
:10373000EA6EEF84668920D0160E6425E96E000ECD
:103740006521EA6E60C3EFFF61C3ECFF62C3ECFF6B
:1037500063C3ECFF1A0E6425E96E000E6521EA6E64
:103760005CC3EFFF5DC3ECFF5EC3ECFF5FC3ECFF28
:10377000000183EC0AF0030104D0000183EC0AF09D
:103780000301E7D064C3E9FF65C3EAFFEF5009080E
:1037900015E1000183EC0AF00D0E03015025E96EDE
:1037A000000E5121EA6EEFA808D065C36CF364C324
:1037B0006BF30001A7EC14F00301CBD064C3E9FF65
:1037C00065C3EAFFEF50040862E1000183EC0AF0F0
:1037D0000D0E03015025E96E000E5121EA6EEFA097
:1037E00045D0100E666F1A0E6425E96E000E652135
:1037F000EA6E010EEF24006E000EEC20016E000E4A
:10380000EC20026E000EEC20ED52ED52ED5200C0A5
:10381000EFFF01C0ECFF02C0ECFFEC6E1A0E642556
:10382000E96E000E6521EA6EEFCF54F3ECCF55F34D
:10383000ECCF56F3ECCF57F30D0E5025E96E000E8A
:103840005121EA6EEFA809D065C36CF364C36BF332
:103850000001A7EC14F008D0030164C3E9FF65C3BD
:10386000EAFF060EEF6E000110D003010D0E502589
:10387000E96E000E5121EA6EEFA806D064C3E9FF9D
:1038800065C3EAFF050EEF6E000162D0030164C359
:10389000E9FF65C3EAFFEF50050840E1000183EC52
:1038A0000AF00D0E03015025E96E000E5121EA6E5B
:1038B000EFA033D0100E666F1A0E6425E96E000E6D
:1038C0006521EA6E010EEF24006E000EEC20016E01
:1038D000000EEC20026E000EEC20ED52ED52ED5287
:1038E00000C0EFFF01C0ECFF02C0ECFFEC6E1A0E4F
:1038F0006425E96E000E6521EA6EEFCF54F3ECCF3C
:1039000055F3ECCF56F3ECCF57F365C36CF364C3B8
:103910006BF30001A7EC14F003011BD064C3E9FFB3
:1039200065C3EAFFEF50060814E1000183EC0AF0DA
:103930000D0E03015025E96E000E5121EA6EEFA82D
:1039400008D065C36CF364C36BF30001A7EC14F0FB
:1039500003010ED0000183EC0AF0100E0301666F24
:103960005FC357F35EC356F35DC355F35CC354F3B3
:10397000665339E0020E5025E96E000E5121EA6EC1
:10398000ECCF6CF3ED52EFCF6BF350C3E9FF51C3B3
:10399000EAFFECCF6EF3ED52EFCF6DF34FC373F34D
:1039A0004EC372F36CC375F36BC374F36EC377F3DA
:1039B0006DC376F35BC37BF35AC37AF359C379F3D0
:1039C00058C378F357C37FF356C37EF355C37DF3D3
:1039D00054C37CF366C380F38169836B826B0001FF
:1039E000C4EC16F003010001C4EF1DF0060E030144
:1039F0002125E96E000E2221EA6EEFCF00F0ECCF18
:103A000001F0ECCF02F0ECCF03F000C03BF301C0BB
:103A10003CF302C03DF303C03EF323C3E9FF24C3DC
:103A2000EAFFEFCF00F0ECCF01F0ECCF02F0ECCFEB
:103A300003F000C03FF301C040F302C041F303C0F4
:103A400042F3436B060E446F26C346F325C345F38A
:103A500046C3CAF345C3C9F30001EBEC0AF002C048
:103A600046F301C045F3030E03014E6F3B0E4D6F4D
:103A70004EC3ADF3AC6FAF6B0C0EAE6F00013FECFD
:103A800011F001C048F30301481F02C049F3491F68
:103A900026C3ABF325C3AAF30001CCEC11F002C09E
:103AA0004BF301C04AF303014B51485D03E14A5116
:103AB000495D07E0000183EC0AF0010E016E6BD056
:103AC00003014F6B4E6B000178EC12F0030E030103
:103AD0004E6F270E4D6F4EC3B9F3B86FBB6B140E0C
:103AE000BA6F0001B9EC0AF0030E0301AB6F270EA9
:103AF000AA6F000196EC12F0030133390F0B006E30
:103B000000360036FC0E00160050EC0F4C6F4C5186
:103B1000255D4D6F000E26594E6F140E4D5D256FBD
:103B2000000E4E59266F33390F0B006E00344D6F67
:103B30004D37FC0E4D174F6B4DC34EF3000178EC23
:103B400012F0030E03014E6F270E4D6F22C350F388
:103B500021C34FF30001A9EF13F001C047F30301A4
:103B60004751FE0813E047C34DF322C34FF321C36F
:103B70004EF3030E516F270E506F26C353F325C328
:103B800052F30001DEEF17F004D00301000183ECD3
:103B90000AF0010E016E68EF3BF0040E0301792577
:103BA000016E000E7A21036E01C07BF37C6F040E60
:103BB0007925E96E000E7A21EA6EECCF7EF3ED52A4
:103BC000EFCF7DF37EC3CAF37DC3C9F30001EBECF5
:103BD0000AF07CC3EAFF7BC3E9FF02C0ECFFED52B1
:103BE00001C0EFFF060E03017925016E000E7A2158
:103BF000036E01C07BF37C6F060E7925E96E000E23
:103C00007A21EA6EECCF7EF3ED52EFCF7DF37EC3E7
:103C1000CAF37DC3C9F30001EBEC0AF07CC3EAFFF1
:103C20007BC3E9FF02C0ECFFED5201C0EFFF020EC3
:103C300003017925016E000E7A21036E01C07BF32A
:103C40007C6F020E7925E96E000E7A21EA6EECCFC8
:103C50007EF3ED52EFCF7DF37EC3CAF37DC3C9F38C
:103C60000001EBEC0AF07CC3EAFF7BC3E9FF02C072
:103C7000ECFFED5201C0EFFF1200030E03017A6F5B
:103C80002D0E796F7AC3B9F3B86FBB6B080EBA6F9C
:103C90000001B9EC0AF00301786B776B28C303F0DD
:103CA00027C3E9FF28C3EAFFEFCF79F37B6B140E3C
:103CB0007A6F7D6B79C37CF300019CEC0FF002C03E
:103CC00076F301C075F3030127C3E9FF28C3EAFFB8
:103CD000080EEF5CEF6E28C303F027C3E9FF28C38B
:103CE000EAFFEFCF79F326C3B9F325C3B8F3BB6B73
:103CF00079C3BAF30001B9EC0AF0030E03017A6F3D
:103D00002D0E796F000149DF030123C3E9FF24C3AE
:103D1000EAFF2DC3EFFF29C3E9FF2AC3EAFF32C33D
:103D2000ECFFED5231C3EFFF2BC3E9FF2CC3EAFFD9
:103D300034C3ECFFED5233C3EFFF7751755D03E100
:103D40007851765D02E0000E01D0010E016E000197
:103D500092EF3BF0010E0301AA6F000173EC0CF02F
:103D600001C075F30301753D01D07CD075C3C3F369
:103D7000C56B140EC46F000187EC0CF0036A0301DD
:103D80002651080F736F000E0320746F2C6B23C332
:103D90002BF32E6B2D6B28C330F327C32FF32AC3CD
:103DA00032F329C331F3030EEA6E330EE96E25C3F5
:103DB000E2FF24C3E1FF2651016E04E0E6CFEEFFEF
:103DC000012EFCD7030E7A6F2B0E796F0001E5DE12
:103DD000080E03012625776B766F22C3ABF321C350
:103DE000AAF3010EAC6F77C3AEF376C3ADF3000157
:103DF00034EC16F0030E0301776F2B0E766F77C34A
:103E0000CFF3CE6F74C3D1F373C3D0F30001EDECE5
:103E10000CF00301C46B140EC36F74C3C6F373C3F9
:103E2000C5F30001C8EC15F002C02EF301C02DF35C
:103E300075C3C3F30301C56B160EC46F000187EC95
:103E40000CF0030E0301776F2D0E766F77C3CFF35F
:103E5000CE6FD16B020ED06F0001EDEC0CF07EEC5A
:103E60000DF003010001C1EF3BF003012C6B216B4E
:103E700021510408D8A035D22151240DF350036AF2
:103E8000610F016E000E032201C026F303C027F369
:103E9000230E2625E96E000E2721EA6EEFB608D024
:103EA000230E2625E96E000E2721EA6EEFA801D029
:103EB00016D226C3E9FF27C3EAFFEF500A0810E035
:103EC00026C3E9FF27C3EAFFEF520BE1230E2625A5
:103ED000E96E000E2721EA6EEF50010B010801E1A7
:103EE000FED126C3E9FF27C3EAFFEF5003080BE129
:103EF000230E2625E96E000E2721EA6EEF50010BF6
:103F0000010801E1ECD100019AEC14F002C025F3A4
:103F100001C024F31F0E03012625E96E000E2721A0
:103F2000EA6EECCF03F0ED52EFCF01F02551035CC8
:103F300004E305E10150245D02E3000E01D0010E0F
:103F4000036A03101BE01F0E2625E96E000E2721D1
:103F5000EA6EECCF03F0ED52EF50FF082D6FFF0E2D
:103F600003542E6F24512D2725512E23010E2D256C
:103F7000016E000E2E21036E015010D01F0E26255B
:103F8000E96E000E2721EA6EECCF03F0ED52EF5000
:103F9000245D006E03502559036E0050226F03C04C
:103FA00023F3210E2625E96E000E2721EA6EECCFC1
:103FB00003F0ED52EFCF01F02351035C05E303E181
:103FC0002251015C01E38BD1010EAA6F000128ECA4
:103FD00015F0015201E185D11F0E03012625016E66
:103FE000000E2721036E01C02DF32E6F00019AEC05
:103FF00014F02EC3EAFF2DC3E9FF02C0ECFFED521F
:1040000001C0EFFF210E03012625E96E000E2721D6
:10401000EA6ED890EF34026EEC34036E0250ED522B
:10402000EF6E03C0ECFF1E0E2625E96E000E272161
:10403000EA6EEF2A26C3E9FF27C3EAFF010EEF5C11
:10404000F70FD8B0C7D0090F000174EF21F0020EAE
:1040500003012C6FBFD01E0E03012625E96E000E52
:104060002721EA6EEF50030803E3120E2C6F16D0DF
:10407000230E2625E96E000E2721EA6EEFA006D05A
:1040800026C3E9FF27C3EAFFEF6A08D0020E2C6FB0
:1040900026C3E9FF27C3EAFF010EEF6E9BD01E0E79
:1040A00003012625E96E000E2721EA6EEF50030872
:1040B00021E30F0E2625E96E000E2721EA6EEF3C64
:1040C00001D013D00F0E2625E96E000E2721EA6ECF
:1040D000EFCF2DF32DC3C3F3C56BC46B000187EC89
:1040E0000CF07EEC0DF004D00301100E2C6F0001DB
:1040F00028D003010F0E2625E96E000E2721EA6E57
:10410000EF3C01D015D00F0E2625E96E000E2721B9
:10411000EA6EEFCF2DF32DC36EF3000102EC00F039
:104120000F0E03012625E96E000E2721EA6EEF68C7
:10413000110E2C6F26C3E9FF27C3EAFF040EEF6EB2
:104140000001030147D01E0E03012625E96E000E73
:104150002721EA6EEF50030803E3010E2C6F08D00D
:1041600027C36CF326C36BF30001A7EC14F0030123
:1041700031D027C36CF326C36BF3A7EC14F0030113
:1041800029D027C36CF326C36BF3A7EC14F003010B
:1041900021D0010E03012C6F26C3E9FF27C3EAFFDC
:1041A000090EEF6E17D01E0E03012625E96E000ED4
:1041B0002721EA6EEF50030803E3010E2C6F08D0AD
:1041C00027C36CF326C36BF30001A7EC14F00301C3
:1041D00001D003012C53D8B482D02CA90FD0160ED5
:1041E0002625E96E000E2721EA6EEFCF28F3ECCFEB
:1041F00029F3ECCF2AF3ECCF2BF31FD0160E262594
:10420000E96E000E2721EA6EEE52EE52EE52EDCF2D
:1042100003F0EDCF02F0EDCF01F0EFCF00F0010E93
:10422000EE26000EEE22EE22ED2203C02BF302C09A
:104230002AF301C029F300C028F3010E2625016EE0
:10424000000E2721036E01C02DF32E6F0B0E2625C5
:10425000E96E000E2721EA6EECCF30F3ED52EFCF7E
:104260002FF30D0E2625E96E000E2721EA6EECCF06
:1042700032F3ED52EFCF31F31A0E2625E96E000E20
:104280002721EA6EEFCF33F3ECCF34F3ECCF35F3E5
:10429000ECCF36F303C073F301C072F330C375F390
:1042A0002FC374F332C377F331C376F32BC37BF39D
:1042B0002AC37AF329C379F328C378F336C37FF38B
:1042C00035C37EF334C37DF333C37CF32CC380F357
:1042D0008169836B826B0001C4EC16F00301212B12
:1042E000C7D50001CDEF3BF0E824F76AF736030F9E
:1042F000F66E430EF7220A00F550FA6E0800F550EC
:10430000F96E4E4056409E40464172417241824194
:104310009241A64103012951240DF3502B6B2A6FC2
:10432000610E2A25E96E000E2B21EA6EEF5003087C
:1043300002E0000E01D0010E016E00011200030127
:104340002951240DF3502B6B2A6F230E2A27000EC0
:104350002B23610E2A25E96E000E2B21EA6E000E3A
:10436000EFB6010E016E0001120003012951240D68
:10437000F350036A610F016E000E032201C02CF39B
:1043800003C02DF3230E2C25E96E000E2D21EA6EBD
:10439000EFA651D0230E2C25E96E000E2D21EA6EDA
:1043A000EFA40ED04F6B140E4E6F000178EC12F09C
:1043B000230E03012C25E96E000E2D21EA6EEF94E9
:1043C000120E2C25E96E000E2D21EA6EECCF2FF394
:1043D000ED52EFCF2EF32E5310E12F530EE10001DB
:1043E00083EC0AF0230E03012C25E96E000E2D212B
:1043F000EA6EEF96000E016E20D0120E2C25E96EAB
:10440000000E2D21EA6EFF0EEF2602E2EE52ED06BF
:104410002BC303F02AC32EF32BC32FF30001B6ECFA
:1044200011F02FC3EAFF2EC3E9FF01C0EFFF010E19
:10443000016E030102D0000E016E0001120036C3AE
:104440003AF335C339F33AC303F0030139C3E9FF43
:104450003AC3EAFFEF5230E038C33CF337C33BF3D3
:104460003CC303F03BC3E9FF3CC3EAFFEF520AE160
:104470003551395D006E36513A59036E00C001F076
:1044800023D010D039C3E9FF3AC3EAFFEFCF3DF3A1
:104490003CC303F03BC3E9FF3CC3EAFFEF503D5D83
:1044A00001E104D03B2BD8B43C2BDAD7392BD8B45C
:1044B0003A2B0001C8D703013551395D006E3651E2
:1044C0003A59036E00C001F00001BCEF22F036C380
:1044D0003AF335C339F33AC303F0030139C3E9FFB3
:1044E0003AC3EAFFEF522AE038C33CF337C33BF349
:1044F0003CC303F03BC3E9FF3CC3EAFFEF5218E0C3
:1045000039C3E9FF3AC3EAFFEFCF3DF33CC303F001
:104510003BC3E9FF3CC3EAFFEF503D5D05E139C312
:1045200001F03AC302F00DD03B2BD8B43C2BE0D7BE
:10453000392BD8B43A2B0001CED70301000E016EFF
:10454000026E0001DDEF22F003012D512E1104E077
:104550002EC303F02D5103D04CC003F04B50316FEC
:1045600003C032F332C336F331C335F330C338F30B
:104570002FC337F3000163D7015003013127000E29
:10458000322332C303F031C3E9FF32C3EAFFEF52F3
:104590000AE14BC0E9FF4CC0EAFF200EEF6E000EAF
:1045A000016E026E27D032C336F331C335F330C308
:1045B00038F32FC337F300018AD702C034F301C0A8
:1045C00033F334C303F0030133C3E9FF34C3EAFF19
:1045D000EF5208E033C3E9FF34C3EAFFEF6A332B3D
:1045E000D8B4342B34C34CF033C34BF031C301F097
:1045F00032C302F000011200030129C3E9FF2AC3FC
:10460000EAFFEFCF2DF32CC303F02BC3E9FF2CC33C
:10461000EAFFEF502D5D15E12AC303F029C3E9FF3E
:1046200003C0EAFFEF5203E1000E016E1FD02AC360
:1046300003F02951292BD8B42A2B2B2BD8B42C2B9F
:10464000DCD72AC303F029C3E9FF2AC3EAFFEFCF6F
:104650002DF32CC303F02BC3E9FF2CC3EAFFEF506B
:104660002D5D02E2FF0E01D0010E016E000112006D
:104670007AC37DF379C37FF378C37EF303017C5360
:1046800003E17B51000816E27FC303F07EC3E9FF1C
:104690007FC3EAFF7D51EF5C05E17EC301F07FC37C
:1046A00002F00BD07E2BD8B47F2B7B51D8B47C0783
:1046B0007B07E5D7000E016E026E000112000301B8
:1046C0007A517C19800B7E6F7AAF05D0791F7A1FE3
:1046D000792BD8B47A2B7CAF05D07B1F7C1F7B2B2A
:1046E000D8B47C2B79517B03F3CF01F0F4CF00F0E9
:1046F0007C03F35000267A517B03F3500020026EB6
:104700007EAF05D0011E021E012AD8B4022A000184
:1047100012000301516B506B300E536F310E546F0A
:10472000320E556F330E566F340E576F350E586F6D
:10473000360E596F370E5A6F380E5B6F390E5C6F3D
:10474000610E5D6F620E5E6F630E5F6F640E606F71
:10475000650E616F660E626F670E636F680E646F41
:10476000690E656F6A0E666F6B0E676F6C0E686F11
:104770006D0E696F6E0E6A6F6F0E6B6F700E6C6FE1
:10478000710E6D6F730E6E6F740E6F6F750E706FAE
:10479000760E716F770E726F780E736F790E746F7D
:1047A0007A0E756F766B46C34BF345C34AF34BC322
:1047B00003F04AC3E9FF4BC3EAFFEF50200804E1CE
:1047C0004A2BD8B44B2BF3D74BC303F04AC3E9FFB2
:1047D0004BC3EAFFEF502D0809E04BC303F04AC377
:1047E000E9FF4BC3EAFFEF502B080BE14BC303F08B
:1047F0004A514A2BD8B44B2BE96E03C0EAFFEF5065
:1048000001D02B0E526F52512D080AE049BF08D03B
:10481000492D01D005D049BF05D04951240802E2F5
:104820000DD184D049534CE0495110081FE14BC3CE
:1048300003F04AC3E9FF4BC3EAFFEF50300816E12B
:10484000010E4A25E96E000E4B21EA6EEF50780802
:1048500009E0010E4A25E96E000E4B21EA6EEF5089
:10486000580804E1020E4A27000E4B23495108085C
:104870000DE14BC303F04AC3E9FF4BC3EAFFEF501E
:10488000300804E1010E4A27000E4B23495102086B
:1048900016E14BC303F04AC3E9FF4BC3EAFFEF50F5
:1048A00030080DE1010E4A25E96E000E4B21EA6E3B
:1048B000EF50620804E1020E4A27000E4B2336D067
:1048C0004BC303F04AC3E9FF4BC3EAFFEF50300884
:1048D00003E00A0E496F2AD0010E4A25E96E000E48
:1048E0004B21EA6EEF50780809E0010E4A25E96E87
:1048F000000E4B21EA6EEF50580807E1100E496F89
:10490000020E4A27000E4B2311D0010E4A25E96EF4
:10491000000E4B21EA6EEF50620806E1020E496F6D
:104920004A27000E4B2302D0080E496F4BC34DF3AC
:104930004AC34CF34BC303F04AC3E9FF4BC3EAFF3E
:10494000EF50300804E14A2BD8B44B2BF3D74BC3BC
:1049500003F04AC3E9FF4BC3EAFFEFCF77F3775188
:10496000400806E277515A0803E37751200901D045
:104970007751776F030E796F530E786F77C37AF3A1
:104980007C6B49C37BF3000173DE02C04FF301C0AF
:104990004EF303014E5302E14F534AE0036A49517B
:1049A000006EE8BE0306776F03C078F351C37AF355
:1049B00050C379F303C07CF37B6F000180DE01C03C
:1049C00077F3530E03014E5D006E030E4F59036ED5
:1049D00000500124016E0250032201C050F303C0B5
:1049E00051F34A2BD8B44B2B4BC303F04AC3E9FF16
:1049F0004BC3EAFFEFCF77F37751400806E27751D8
:104A00005A0803E37751200901D07751776F030EDD
:104A1000796F530E786F77C37AF37C6B49C37BF35E
:104A2000000126DE02C04FF301C04EF3B2D70301EE
:104A30004A514C5D13E14B514D5D10E14751481116
:104A400009E047C3E9FF48C3EAFF46C3ECFFED5264
:104A500045C3EFFF000E016E026E10D047514811A2
:104A600009E047C3E9FF48C3EAFF4BC3ECFFED523F
:104A70004AC3EFFF50C301F051C302F0000113EF2E
:104A800026F04DC34FF34CC34EF34FC303F0030165
:104A90004EC3E9FF4FC3EAFFEF5206E04E2BD8B4F6
:104AA0004F2B0001F2D703014C514E5D006E4D516A
:104AB0004F59036E00C001F00001120049C34FF3CB
:104AC00048C34EF34BC351F34AC350F30301515152
:104AD0004F5D3EE303E14E51505D3AE24C515025AB
:104AE000016E4D515121036E4F51035C31E303E1DF
:104AF00001504E5D2DE24C514E274D514F234C51EC
:104B000050274D5151234D5303E14C5100081FE2F2
:104B10004E51D8B44F074E074EC352F34FC353F311
:104B20005051D8B45107500751C303F050C3E9FFA7
:104B300051C3EAFFEFCF54F34FC3EAFF4EC3E9FF7F
:104B400054C3EFFF4C51D8B44D074C07DCD724D0E9
:104B50004D5303E14C5100081FE24FC303F04E5187
:104B60004E2BD8B44F2B526F03C053F351C303F0F5
:104B70005051502BD8B4512BE96E03C0EAFFEFCF50
:104B800054F353C3EAFF52C3E9FF54C3EFFF4C5140
:104B9000D8B44D074C07DCD748C301F049C302F035
:104BA00000013DEF26F00301426B3DC33FF33CC3E0
:104BB0003EF33DC303F03CC3E9FF3DC3EAFFEFCF43
:104BC00043F3435361E043512B080CE13DC303F031
:104BD0003C513C2BD8B43D2BE96E03C0EAFF200EBC
:104BE000EF6E50D0435125084AE1010E3C25456F38
:104BF000000E3D21466F030EEA6E400EE96E46C37D
:104C0000E2FF45C3E1FF020E016EE6CFEEFF012E8B
:104C1000FCD7030E466F400E456F486B476B100E76
:104C2000496F000176D501C044F303013DC303F091
:104C30003C513C2BD8B43D2BE96E03C0EAFF44C382
:104C4000EFFF020E3C25456F000E3D21466F3DC330
:104C50004DF33CC34CF3000114DF010E015C030172
:104C6000476F3DC349F33CC348F346C34BF345C3C9
:104C70004AF34D6B4C6F000121D704D003013C2B4C
:104C8000D8B43D2B030195D73EC301F03FC302F0DA
:104C900000011200030145C3E9FF46C3EAFFEFCF5D
:104CA00049F348C303F047C3E9FF48C3EAFFEF50A5
:104CB000495D48E046C303F045C3E9FF46C3EAFF48
:104CC000EFCF49F34951400803E249515A0806E23F
:104CD000495160084CE249517A0849E348C303F05E
:104CE00047C3E9FF48C3EAFFEFCF49F34951400802
:104CF00003E249515A0806E24951600838E2495135
:104D00007A0835E345C3E9FF46C3EAFFEFCF49F32D
:104D100048C303F047C3E9FF48C3EAFF200EEF246E
:104D2000495D10E047C3E9FF48C3EAFFEFCF49F30D
:104D300046C303F045C3E9FF46C3EAFF200EEF2454
:104D4000495D15E146C303F045C3E9FF46C3EAFFE9
:104D5000EF5203E1000E016E1FD046C303F0455130
:104D6000452BD8B4462B472BD8B4482B94D746C3F1
:104D700003F045C3E9FF46C3EAFFEFCF49F348C359
:104D800003F047C3E9FF48C3EAFFEF50495D02E281
:104D9000FF0E01D0010E016E000112000301306B05
:104DA0002F6B2E6B2D6B2CC346F32BC345F3020EDA
:104DB000486FFD0E476F00016DDF01520AE1010EE1
:104DC000036EB00E03012D6F03C02EF32F6B306BFB
:104DD00000012CC346F32BC345F3020E0301486FB9
:104DE0004769000157DF01520AE1050E036EC20E4A
:104DF00003012D6F03C02EF32F6B306B00012DC309
:104E000000F02EC301F02FC302F030C303F08EEF89
:104E100036F0006A016A03014C51D8904DB100266A
:104E2000003201324DB30026003201324DB500266A
:104E3000003201324DB70026003201324DB9002652
:104E4000003201324DBB0026003201324DBD00263A
:104E5000003201324DBF002600320132000199EFCD
:104E600027F003014A6B486B0A0E496F476B4551A7
:104E7000461103E1000E016EBBD04A514A2B452575
:104E8000E96E000E4621EA6EEFCF4BF34B512D0831
:104E90000CE1010E486F4A514A2B4525E96E000E80
:104EA0004621EA6EEFCF4BF30CD04B512B0809E1B2
:104EB0004A514A2B4525E96E000E4621EA6EEFCF96
:104EC0004BF34B512F08D8B08BD04B513908D8A099
:104ED00087D04B5130081EE14A514525E96E000E3E
:104EE0004621EA6EEF50780809E04A514525E96EFF
:104EF000000E4621EA6EEF5058080CE1100E496F83
:104F00004A2B4A514A2B4525E96E000E4621EA6E8E
:104F1000EFCF4BF349510A081CE14B512F0818E21F
:104F20004B51390815E30A0E4C6F47C34DF300018E
:104F300070D7300E03014B5D0124476F4A514A2B55
:104F40004525E96E000E4621EA6EEFCF4BF3E5D71B
:104F500047D04951100844E14B51600806E24B51DB
:104F60007A0803E34B51DF0B01D04B514B6F4B5190
:104F70002F0803E24B51390806E24B51400830E25A
:104F80004B5146082DE34B512F080CE24B51390889
:104F900009E347394C6FF00E4C17300E4B5D4C2532
:104FA000476F09D047394C6FF00E4C17410E4B5DDF
:104FB0000A0F4C25476F4A514A2B4525E96E000ED2
:104FC0004621EA6EEFCF4BF34B51600806E24B519E
:104FD0007A0803E34B51DF0B01D04B514B6FC7D71E
:104FE000482D04D049510A0801E1476D47C301F03B
:104FF0000001120041C346F340C345F3030E030111
:10500000486F070E476F000145DE015216E143C3AA
:1050100046F342C345F325DF01C044F30301445383
:1050200007E092948984010E0201F76F05D0030115
:10503000929489940201F76B000141C346F340C387
:1050400045F3030E0301486F110E476F000122DE86
:1050500001521CE143C346F342C345F302DF01C0E2
:1050600044F3F250006EF29EA96A44C3A8FFA69CC6
:10507000A69EA6840F01550EA76EAA0EA76EA68245
:10508000A6B2FED7A6940050F212000141C346F327
:1050900040C345F3030E0301486F0C0E476F000138
:1050A000F9DD01521DE143C346F342C345F3D9DEA6
:1050B00001C044F3F250006EF29E010EA96E44C38B
:1050C000A8FFA69CA69EA6840F01550EA76EAA0E49
:1050D000A76EA682A6B2FED7A6940050F2120001D7
:1050E00041C346F340C345F3030E0301486F140E5A
:1050F000476F0001CFDD01521CE143C346F342C3B9
:1051000045F3AFDE01C044F3F250006EF29E030E91
:10511000A96E44C3A8FFA69CA69EA6840F01550EA7
:10512000A76EAA0EA76EA682A6B2FED7A6940050BE
:10513000F2120001CFEF28F036C338F335C337F34E
:1051400003013A6B396B35C3E9FF36C3EAFFEFCF92
:105150003BF33B51260802E03B532EE135C3E9FF08
:1051600036C3EAFFEF6A38C33DF337C33CF30001AF
:105170001ADD3AC33DF339C33CF315DD34C33FF3C5
:1051800033C33EF332C33DF331C33CF338C341F381
:1051900037C340F33AC343F339C342F32BD7010E6D
:1051A00003013525376F000E3621386F3A6B396BA6
:1051B0003B5301E113D00ED03B513D080BE135C309
:1051C000E9FF36C3EAFFEF6A010E3525396F000E9D
:1051D00036213A6F352BD8B4362BB5D700011200E3
:1051E0000301316B2F6B0A0E306F2E6B2D6B2B5121
:1051F0002C1104E1000E016E026EE3D03151312B0F
:105200002B25E96E000E2C21EA6EEFCF32F33251DE
:105210002D080CE1010E2F6F3151312B2B25E96E3A
:10522000000E2C21EA6EEFCF32F30CD032512B0856
:1052300009E13151312B2B25E96E000E2C21EA6E4C
:10524000EFCF32F332512F08D8B0ADD032513908F8
:10525000D8A0A9D0325130081EE131512B25E96E7A
:10526000000E2C21EA6EEF50780809E031512B2511
:10527000E96E000E2C21EA6EEF5058080CE1100E7A
:10528000306F312B3151312B2B25E96E000E2C2143
:10529000EA6EEFCF32F330510A0823E132512F0882
:1052A0001FE2325139081CE37A6B0A0E796F2EC364
:1052B0007CF32DC37BF300015FEC23F0300E030180
:1052C000325D01242D6F000E02202E6F3151312BE3
:1052D0002B25E96E000E2C21EA6EEFCF32F3DED7DC
:1052E00062D0305110085FE13251600806E232515D
:1052F0007A0803E33251DF0B01D03251326F325161
:105300002F0803E23251390806E2325140084BE2DD
:105310003251460848E332512F081AE23251390817
:1053200017E32D35336F2E35346F3337343733373A
:10533000343733373437F00E3317300E325D3325C0
:10534000016E000E3421036E01C02DF32E6F16D0B6
:105350002D35336F2E35346F333734373337343799
:1053600033373437F00E3317410E325D0A0F3325D1
:10537000016E000E342101C02DF32E6F3151312BFF
:105380002B25E96E000E2C21EA6EEFCF32F332515D
:10539000600806E232517A0803E33251DF0B01D094
:1053A0003251326FACD730510A0807E12F2D05D0AA
:1053B0002D1F2E1F2D2BD8B42E2B2DC301F02EC345
:1053C00002F000011CEF37F003012C51240DF350C3
:1053D000036A610F016E000E032201C02DF303C0AA
:1053E0002EF3230E2D25E96E000E2E21EA6EEFB668
:1053F00003D0000E016E0DD0000183EC0AF0230EE5
:1054000003012D25E96E000E2E21EA6EEF96010EA6
:10541000016E0001120003014C51240DF3504E6B3C
:105420004D6F140E4D25016E000E4E21036E01507E
:10543000610FE96E000E0320EA6EECCF4EF3ED52E1
:10544000EFCF4DF34D5305E14E5303E1000E016ED6
:105450002ED04C51240DF3504E6B4D6F0F0E4D2539
:10546000016E000E4E21036E0150610FE96E000EB9
:105470000320EA6EEF3C08D0AA6B000128EC15F07F
:105480000150030114D013D04C51240DF3504E6B36
:105490004D6F230E4D27000E4E23610E4D25E96EF4
:1054A000000E4E21EA6E000EEFB2010E016E0001F9
:1054B000120039C324F161EF32F003015E51240D73
:1054C000F350036A610F016E000E032201C05FF307
:1054D00003C060F30F0E5F25E96E000E6021EA6ED7
:1054E000EF3C03D0000E016ECBD0230E5F25E96E9A
:1054F000000E6021EA6EEFCF00F00030010B03E1F7
:10550000000E016EBDD0010E5F25016E000E602100
:10551000036E01C061F3626F0B0E5F25E96E000E32
:105520006021EA6EECCF64F3ED52EFCF63F30D0E22
:105530005F25E96E000E6021EA6EECCF66F3ED5256
:10554000EFCF65F3160E5F25E96E000E6021EA6E5F
:10555000EFCF67F3ECCF68F3ECCF69F3ECCF6AF3EE
:105560001A0E5F25E96E000E6021EA6EEFCF6BF335
:10557000ECCF6CF3ECCF6DF3ECCF6EF30F0E5F2539
:10558000E96E000E6021EA6EEFCF6FF3100E5F251B
:10559000E96E000E6021EA6EECCF71F3ED52EFCFB1
:1055A00070F303C073F301C072F364C375F363C394
:1055B00074F366C377F365C376F36AC37BF369C399
:1055C0007AF368C379F367C378F36EC37FF36DC36F
:1055D0007EF36CC37DF36BC37CF3180E806F6FC3D7
:1055E00081F371C383F370C382F30001C4EC16F03E
:1055F000160E03015F25016E000E6021036E01C0CF
:1056000061F3626FEA6E01C0E9FFEFCF63F3ECCFA5
:1056100064F3ECCF65F3ECCF66F3100E5F25E96E13
:10562000000E6021EA6EECCF03F0ED52EFCF00F0F8
:1056300003C001F0026A036A63510026645101222B
:10564000655102226651032262C3EAFF61C3E9FF8A
:1056500000C0EFFF01C0ECFF02C0ECFF03C0ECFF95
:10566000230E5F25E96E000E6021EA6EEF92230E95
:105670005F25E96E000E6021EA6EEF98010E016E63
:105680000001120003015851240DF350036A610F09
:10569000016E000E032201C05AF303C05BF3140E27
:1056A0005A25E96E000E5B21EA6EECCF5FF3ED52F6
:1056B000EFCF5EF35E5305E15F5303E1000E016E31
:1056C00081D00F0E5A25E96E000E5B21EA6EEF3C89
:1056D00039D00F0E5A25016E000E5B21036E01C0FA
:1056E0005EF35F6FAA6B000173EC0CF05FC3EAFF1F
:1056F0005EC3E9FF01C0EFFF0F0E03015A25E96EFB
:10570000000E5B21EA6EEF3C03D0000E016E5AD012
:10571000100E5A25E96E000E5B21EA6EEC6AED521E
:10572000EF6A0F0E5A25E96E000E5B21EA6EEFCF8D
:105730005EF35EC3C3F3C56B280EC46F000187EC34
:105740000CF00301230E5A25E96E000E5B21EA6E70
:10575000EF8859C3CDF30001DEEC0CF0140E030109
:105760005A25E96E000E5B21EA6EFF0EEF2602E27B
:10577000EE52ED06100E5A25E96E000E5B21EA6E20
:10578000ECCF5DF3ED52EFCF5CF35C2BD8B45D2B27
:10579000100E5A25E96E000E5B21EA6E5DC3ECFF28
:1057A000ED525CC3EFFF5D5102080AE2FF0A03E11C
:1057B0005C51C90805E258C35EF300017EDE0301B7
:1057C000010E016E0001EAEF2BF024C158F357C31C
:1057D00059F358D7015012000900F6CF3AF3F7CF2A
:1057E0003BF3F5CF57F3F1DF3AC3F6FF3BC3F7FFC7
:1057F0000301392F01D002D00001EED70001ACEF38
:1058000032F0EACF41F3E9CF40F303013A39F0092E
:105810003C6F3C27E20F3D6F320F3F6F3A510F0B49
:105820003D273D273F27E90F3E6F3E273E27393969
:105830000F0B3E273F273E373F373F1F3F3739513A
:105840000F0B3F273C37070E3B6F0A0E3E073F27E3
:10585000FDE33D073E27FDE33C073D27FDE33B0716
:105860003C27FDE3030EEA6E3B0EE96E070E401582
:10587000409DE926000EEA22E9503F0804E1EA5083
:10588000030801E1408DEF50006E08E140BD06D0F5
:1058900040B915D040B702D0200E03D040874099C0
:1058A000300E0026EACF3AF3E9CF39F300C057F3C0
:1058B00000018BDF3AC3EAFF39C3E9FF0301EE5071
:1058C00040ADDAD70001B4EF32F00900F5520CE038
:1058D000F6CF39F3F7CF3AF3F5CF57F376DF39C385
:1058E000F6FF3AC3F7FFF1D71200EF520FE0EACF0D
:1058F0003AF3E9CF39F3EFCF57F367DF3AC3EAFF63
:1059000039C3E9FFE92AD8B4EA2AEFD70FEF33F019
:1059100047C34CF380DD015204E1000E016E026EBC
:1059200072D003014751240DF3504D6B4C6F0F0E95
:105930004C25016E000E4D21036E0150610FE96E82
:10594000000E0320EA6EEF3C03D0496B486B16D083
:105950004751240DF3504D6B4C6F100E4C25016ECA
:10596000000E4D21036E0150610FE96E000E032001
:10597000EA6EECCF49F3ED52EFCF48F3CA0ED88070
:1059800048554A6F030E49554B6F4751240DF3504C
:105990004D6B4C6F140E4C25016E000E4D21036EA5
:1059A0000150610FE96E000E0320EA6EECCF03F0A8
:1059B000ED52EFCF01F003504B5D1AE303E14A5182
:1059C000015C16E24751240DF3504D6B4C6F140EE1
:1059D0004C25016E000E4D21036E0150610FE96EE2
:1059E000000E0320EA6EECCF03F0ED52EF5003D02F
:1059F0004BC303F04A514A6F03C04BF34AC301F053
:105A00004BC302F00001120003013BC3E9FF3CC39A
:105A1000EAFFECCF03F0ED52EFCF41F303C042F3C6
:105A200042C34DF341C34CF3000141EC25F00301A7
:105A3000406B01C03FF33F51401103E1000E016E86
:105A400042D024C147F3000163DF02C03EF301C02E
:105A50003DF303013D513E1103E1010E016E33D0D0
:105A60003E51405D07E303E13F513D5D03E2010E1E
:105A7000436F05D040C33EF33FC33DF3436B3EC38A
:105A800003F03D51D8B43E073D07031011E042C377
:105A900003F04151412BD8B4422BE96E03C0EAFF19
:105AA000EFCF44F344C357F300018FDE0301E7D780
:105AB0003BC3E9FF3CC3EAFF42C3ECFFED5241C3E5
:105AC000EFFF43C301F0000112005CC301F05BC3B0
:105AD00000F00066012A0900F5CFEEFF002EFBD78B
:105AE000012EF9D7F86A120003014F6B4E6B5681F5
:105AF00049C3E9FF4AC3EAFFECCF51F3ED52EFCFC0
:105B000050F347C3E9FF48C3EAFFEFCF52F3ECCFAE
:105B100053F3ECCF54F3ECCF55F355C303F054C318
:105B200002F053C301F052C300F0010E5227D8B067
:105B3000532BD8B4542BD8B4552B03C05AF302C0FE
:105B400059F301C058F300C057F302C0F8FF01C079
:105B5000F7FF00C0F6FF030EEA6E4C0EE96E5C6BB9
:105B6000010E5B6F0001B1DF03014C51250841E1DB
:105B700055C303F054C302F053C301F052C300F005
:105B8000010E5227D8B0532BD8B4542BD8B4552B70
:105B900003C05AF302C059F301C058F300C057F3D1
:105BA00002C0F8FF01C0F7FF00C0F6FF030EEA6E67
:105BB0004D0EE96E5C6B010E5B6F000186DF030129
:105BC0004D51250814E14F51515D0FE303E1505150
:105BD0004E5D0BE24B5305E0250E576F0001F5DDDE
:105BE00003014E2BD8B44F2B01D01CD001D01AD0BA
:105BF00018D04C5314E04F51515D0FE303E1505165
:105C00004E5D0BE24B5305E04CC357F30001DDDD65
:105C100003014E2BD8B44F2B01D004D002D05691A3
:105C200001D07BD756A108D0FF0E5227D8A053270A
:105C3000D8A05427D8A0552749C3E9FF4AC3EAFF93
:105C40004FC3ECFFED524EC3EFFF47C3E9FF48C31C
:105C5000EAFF52C3EFFF53C3ECFF54C3ECFF55C33D
:105C6000ECFF4CC301F0000112000301436B426BD7
:105C700024C147F300014CDE02C045F301C044F3E8
:105C800003014451451103E1010E016E4ED03BC3A7
:105C9000E9FF3CC3EAFFEFCF3EF3ECCF3FF3ECCF9D
:105CA00040F3ECCF41F343694269030E486F3E0E67
:105CB000476F030E4A6F420E496F4B6B000114DFB2
:105CC00001C03DF303014251431106E13D51250856
:105CD00003E0000E016E29D04551435D0BE303E163
:105CE0004251445D07E245C343F344C342F3010E0E
:105CF000466F0CD03D51250803E1020E466F06D0D9
:105D00003D5303E0010E466F01D0466B3CC348F3A0
:105D10003BC347F3030E4A6F420E496F010E4B6FB0
:105D20000001E2DE030146C301F0000161EF33F040
:105D30003FC3F8FF3EC3F7FF3DC3F6FF030EEA6E15
:105D4000410EE96E03015C6B010E5B6F0001BDDE6D
:105D5000030141C301F0000184EF33F006C3EAFF01
:105D600005C3E9FF030159C3EFFFE92AD8B4EA2AC2
:105D7000EF6A052BD8B4062B000112000900F5527A
:105D80000CE0F6CF4CF3F7CF4DF3F5CF59F3E6DF48
:105D90004CC3F6FF4DC3F7FFF1D71200016603D0E5
:105DA000026602D007D0022A00C0EEFF012EFCD707
:105DB000022EFAD7120003015951D8B471D0006EE7
:105DC0005D51D8B46DD0002604E3810E002668E250
:105DD00004D07F0E005E64E363E05AC361F35E515A
:105DE000611B5A8F5E8F5C516003F4CF63F35B518C
:105DF0005F03F4CF03F0F3CF62F36003F350632744
:105E0000F4506223000E03225C515F03F3506327BA
:105E1000F4506223000E026A032202225A516003E8
:105E2000F3506227F4500322000E02225A515F03FE
:105E3000F3500326F4500222000E016A01225C5145
:105E40005E03F3506227F4500322000E0222012267
:105E50005B515E03F3500326F4500222000E012230
:105E60005A515E03F3500226F4500122002A01BE6B
:105E700005D062370336023601360006000E62AFE7
:105E80000AD0032A02220122015005E1025003E157
:105E9000035001E1002A61BF018E61AF019E04D071
:105EA000006A016A026A036A0001D9EF2FF0030158
:105EB0005951B608596F036A5AC35DF35A8FD89087
:105EC0005A335B335C330332023201320032592FD2
:105ED000F6D75DAF0BD0001E011E021E031E002A66
:105EE000D8B4012AD8B4022AD8B4032A0001EEEFAC
:105EF0002FF0D8B204D0030EEA6E610EE96E006A8C
:105F0000016A026A036A0301616B626B636B646B13
:105F100060515F115E115D112CE0200E656FD8900D
:105F200059375A375B375C376137623763376437C5
:105F30006051645D08E15F51635D05E15E51625D42
:105F400002E15D51615D0FE35D51615F5E51D8A07B
:105F50005E3D625F5F51D8A05F3D635F6051D8A036
:105F6000603D645FD8800036013602360336652F07
:105F7000D6D761C3EFFF62C3ECFF63C3ECFF64C31A
:105F8000ECFF00011200E9500301516F5051536FB3
:105F90001BE04FC35CF34EC35BF34DC35AF34CC3DA
:105FA00059F3606B5F6B200E5E6F820E5D6F0001B8
:105FB00002D703C04FF302C04EF301C04DF300C03F
:105FC0004CF30301532FE5D74FC35CF34EC35BF390
:105FD0004DC35AF34CC359F3000169D703C04FF3C3
:105FE00002C04EF301C04DF300C04CF303014FAFAC
:105FF0000DD05107518B4C1F4D1F4E1F4F1F4C2B67
:10600000D8B44D2BD8B44E2BD8B44F2B3B0E586F71
:106010009A0E576FCA0E566F556B0A0E536F50513A
:10602000D8B4512BD882030EEA6E4C0EE96E4FC3E2
:106030005CF34EC35BF34DC35AF34CC359F358C3DF
:1060400060F357C35FF356C35EF355C35DF30001BE
:1060500050DF0150005213E103015029535DD8A4D1
:1060600002D000010CD051510DE00F0B535D01E047
:1060700040E251BF3ED051BD05D0200E34D0200E9D
:106080000301511751AB0ED0519B5051D8A4510769
:106090000050516F2D0E596F000160DE0301515108
:1060A000006E516B5051535D0CE10050516F2E0E3C
:1060B000596F000153DE03015151006E200E51173C
:1060C000000E300E51AB0FD0519B5051D8A4510748
:1060D0000050516F2D0E596F000140DE03015151E8
:1060E000006E516B300E002600C059F3000136DE01
:1060F0000301D89258C35CF357C35BF356C35AF3FA
:1061000055C359F3606B5F6B5E6B0A0E5D6F0001E8
:10611000F0DE03C058F302C057F301C056F300C0CD
:1061200055F30301532F7ED700018CEF31F00301AB
:106130005551016A545D03E254C300F00CD0006A6B
:10614000080E566F543700365551005CD8B0006EBB
:106150000136562FF7D700011200200E03014FA978
:10616000300E506F4EC300F04EAF08D0001E002A14
:1061700000C04EF32D0E506F4F8F4F8101504EC314
:1061800054F3640E556F0001D2DF00C04EF3300EA1
:1061900001240301516F4EC354F30A0E556F0001E1
:1061A000C6DF300E00240301536F300E0124526FFE
:1061B00050C300F0300E515D04E04F834FBF4F8558
:1061C00012D050C351F3200E506F300E525D04E0D8
:1061D0004F814FBF4F8307D0D8A44F8104E151C3F3
:1061E00052F3200E516F4FB505D04FB307D04FB1CA
:1061F00009D00CD050C359F30001B0DD51C359F39D
:106200000001ACDD52C359F30001A8DD53C359F3BB
:106210000001A4DD12000301416B426B436B446B30
:10622000456B466B476B486B496B4A6B4B6B3FC387
:10623000EAFF3EC3E9FFE26AE16A4051016E04E011
:10624000E6CFEEFF012EFCD7300E3D5DF90FD8B042
:10625000FBD0070F00013EEF32F00201F7530DE1D2
:10626000030E0301066F410E056F080EF66E060E53
:10627000F76E000183DD0BD00201030EEA6E410EC2
:10628000E96E006A026A0A0E016E000187DD030EE4
:1062900003014D6F410E4C6F000141EC25F001C030
:1062A0004BF30301D1D00201F72D0DD0030E0301F2
:1062B000066F410E056F100EF66E060EF76E0001AA
:1062C0005DDD0BD00201030EEA6E410EE96E006A3D
:1062D000026A0A0E016E000161DD030E03014D6FBB
:1062E000410E4C6F000141EC25F001C04BF303015E
:1062F000ABD0030E0301066F410E056F890EE96EE8
:10630000FBC24FF3FAC24EF3F9C24DF3F8C24CF39D
:10631000020E506F000137D6030E03014D6F410E80
:106320004C6F000141EC25F001C04BF303018CD010
:10633000F2CF4CF3F29EA96AA69CA69EA680A85016
:1063400003014CBFF28E4D6F030E066F410E056FB9
:106350004DC34EF3180E4F6F0001FFDE030E030115
:106360004D6F410E4C6F000141EC25F001C04BF325
:1063700003016AD0F2CF4CF3F29E010EA96EA69CE7
:10638000A69EA680A85003014CBFF28E4D6F030E4F
:10639000066F410E056F4DC34EF3180E4F6F00018F
:1063A000DCDE030E03014D6F410E4C6F000141EC2A
:1063B00025F001C04BF3030147D0F2CF4CF3F29E1E
:1063C000030EA96EA69CA69EA680A85003014CBFF2
:1063D000F28E4D6F030E066F410E056F4DC34EF3E7
:1063E000180E4F6F0001B9DE030E03014D6F410E11
:1063F0004C6F000141EC25F001C04BF3030124D0A8
:106400000201FC2D0BD0030E0301066F410E056F38
:10641000310E596F0001A2DC0AD00201030E030104
:10642000066F410E056F300E596F000197DC030EA9
:1064300003014D6F410E4C6F000141EC25F001C08E
:106440004BF3030101D003014B5313E04B51405D6B
:10645000D8A040C34BF33FC3EAFF3EC3E9FF030E9E
:10646000E26E410EE16E0A0E016EE6CFEEFF012EE6
:10647000FCD74BC301F00001B7EF33F0E824F76A13
:10648000F736970FF66E640EF7220A00F550FA6E93
:106490000800F550F96E5A62A662F26230637463C6
:1064A000BA630064036A03012D51210FE96E010EE6
:1064B0000320EA6EEFCF36F336C339F3000159EF0C
:1064C0002AF003012D51040DF350036A250FE96EE4
:1064D000010E0320EA6EEFCF39F3ECCF3AF3ECCFA5
:1064E0003BF3ECCF3CF33953D8A4A0D03A53D8A413
:1064F0009DD03B53D8A49AD03C53D8A497D0036ADC
:106500002DC302F0D890023603360250290FE96EEF
:10651000010E0320EA6EEC6AED52EF6A2D51040D74
:10652000F350036A250FE96E010E0320EA6E30C3B3
:10653000EFFF31C3ECFF32C3ECFF33C3ECFF010EBE
:106540000101536F680EF66E010EF76E090E03011E
:10655000396F0001ECEF2BF0100EE96E2FC33AF308
:106560002EC339F301EF2CF0200E0301576F000109
:10657000E5EC2BF003012E51006E2F51036E0350FA
:1065800005E1C80E005C000112E00301010E035C8E
:1065900005E1940E005C000117E00301010E035CAD
:1065A00005E1F40E005C000116E003011CD04F0E63
:1065B0000301576F0001E5EC2BF04B0E0301576F01
:1065C0000001E5EC2BF010D0760EF66E010EF76EA2
:1065D00065EC2CF009D0800EF66E010EF76E65ECBE
:1065E0002CF002D0030100018E0EF66E010EF76E44
:1065F00065EC2CF00301345135110AE035C3EAFF94
:1066000034C3E9FF000175EF2CF0000108D003014D
:10661000A00EF66E010EF76E000165EC2CF0AA0ECE
:10662000F66E010EF76E65EC2CF00301036A2DC3C4
:1066300002F0D890023603360250290FE96E010E9F
:106640000320EA6EEF5226E0036A2DC302F0D890D1
:10665000023603360250290F016E010E032201C0DB
:1066600039F303C03AF303C03CF301C03BF300012C
:1066700004EC2DF0036A03012DC302F0D89002361A
:1066800003360250290FE96E010E0320EA6EEC6A10
:10669000ED52EF6A0101532DB2D003012D51040DCB
:1066A000F350036A250F016E010E032201C039F376
:1066B00003C03AF303C03CF301C03BF3000135EFE4
:1066C0002EF001C037F3030137510208D8A48ED051
:1066D0002D51040DF350036A250FE96E010E0320BE
:1066E000EA6EEFCF39F3ECCF3AF3ECCF3BF3ECCFDC
:1066F0003CF33CC340F33BC33FF33AC33EF339C3DF
:106700003DF3000198EF2EF001C038F303012D5145
:10671000040DF350036A250FE96E010E0320EA6EA3
:10672000010EEF24006E000EEC20016E000EEC2036
:10673000026E000EEC20ED52ED52ED5200C0EFFF64
:1067400001C0ECFF02C0ECFFEC6E33C33CF332C37C
:106750003BF331C33AF330C339F338C33DF3010E91
:106760003F6F2B0E3E6F270E406F000154D5036A1A
:1067700003012DC302F0D890023603360250290FD0
:10678000E96E010E0320EA6E010EEC6EED522B0E47
:10679000EF6E036A2DC302F0D89002360336025022
:1067A000290F016E010E032201C039F303C03AF331
:1067B00003C03CF301C03BF3000104EC2DF001C029
:1067C00037F30301375310E1036A2DC302F0D89069
:1067D000023603360250290FE96E010E0320EA6EDD
:1067E000EC6AED52EF6A01D009D007D0375304E1CB
:1067F000020E0101536F030101D050D70101535123
:10680000020802E1030E536F36C35EF300015DEC34
:106810002AF001015351030802E0000E01D0010EDD
:10682000016E0001120003012951240DF350036A87
:10683000610F016E000E032201C02AF303C02BF387
:106840002AC3E9FF2BC3EAFFEF50030810E02AC375
:10685000E9FF2BC3EAFFEF50020809E02BC36CF3FA
:106860002AC36BF30001A7EC14F079D0030129C30C
:106870002CF30001E4EC29F0010E03012A25016E3E
:10688000000E2B21036E01C02CF32D6F0B0E2A2559
:10689000E96E000E2B21EA6EECCF2FF3ED52EFCF15
:1068A0002EF30D0E2A25E96E000E2B21EA6EECCF99
:1068B00031F3ED52EFCF30F3160E2A25E96E000EBC
:1068C0002B21EA6EEFCF32F3ECCF33F3ECCF34F37E
:1068D000ECCF35F31A0E2A25E96E000E2B21EA6E55
:1068E000EFCF36F3ECCF37F3ECCF38F3ECCF39F30F
:1068F00003C073F301C072F32FC375F32EC374F397
:1069000031C377F330C376F335C37BF334C37AF303
:1069100033C379F332C378F339C37FF338C37EF3DB
:1069200037C37DF336C37CF3110E806F8169836BAF
:10693000826B0001C4EC16F0160E03012A25E96EE5
:10694000000E2B21EA6E010EEE26000EEE22EE2244
:10695000ED222AC3E9FF2BC3EAFF040EEF6E00010C
:10696000CFEF3AF00301276B2753D8A4E5EF3AF0B5
:10697000D8902735036A220FE96E010E0320EA6ED4
:10698000ECCF2AF3ED52EFCF29F3293D04D02A535F
:1069900002E1E5EF3AF0036A2751210FE96E010E9B
:1069A0000320EA6EEFCF28F328C329F300018AEC15
:1069B00021F001520EE1D89003012735036A220F1E
:1069C000E96E010E0320EA6E010EEC6EED52EF6EE1
:1069D0000001D89003012735036A220FE96E010EEA
:1069E0000320EA6EEF50006EEE52ED50036E010E82
:1069F000035C05E1010E005C000158E00301010E9B
:106A0000035C05E1020E005C000158E00301010E89
:106A1000035C06E1030E005C0001D8B4A7D00301BB
:106A2000010E035C06E1040E005C0001D8B4CFD275
:106A30000301010E035C06E1050E005C0001D8B401
:106A4000F5D20301010E035C07E1060E005C0001B4
:106A5000D8B476EF39F00301010E035C07E1070EAD
:106A6000005C0001D8B497EF39F00301010E035C1C
:106A700007E1080E005C0001D8B43DEF3AF00301D5
:106A8000010E035C07E1090E005C0001D8B462EF5F
:106A90003AF00301010E035C07E10A0E005C0001FD
:106AA000D8B4DFEF3AF00301E0EF3AF028C329F35E
:106AB0008AEC21F0015202E1E1EF3AF003012751A3
:106AC000FE0DF3502A6B296F710E2925E96E010E18
:106AD0002A21EA6EEF6A036A27516F0FE96E020EF0
:106AE0000320EA6EEF6AD8902735036A220FE96E19
:106AF000010E0320EA6E010EEC6EED52030EEF6EF6
:106B0000D8902735036A770F016E020E032201C069
:106B100029F303C02AF300019AEC14F02AC3EAFF18
:106B200029C3E9FF02C0ECFFED5201C0EFFF0301F2
:106B30002751040DF350036A710FE96E020E032012
:106B4000EA6EEE52EE52EC6AED52EF6AED52EF6AE7
:106B5000ED52EF6AD8902735036A750FE96E020E81
:106B60000320EA6EEC6AED52EF6A00010301219303
:106B700028C329F300019FEC21F00152D8B4A9D118
:106B800028C329F3030E03012B6F220E2A6F000185
:106B9000B5EC21F00152D8B49CD1030122511F0859
:106BA00025E2036A27516F0FE96E020E0320EA6E99
:106BB000EF50FB081BE32751FE0DF3502A6B296FA2
:106BC000036A27516F0FE96E020E0320EA6EEF5041
:106BD000EF2A036A2925016E2A5103220150710F01
:106BE000E96E010E0320EA6E22C3EFFF22510A086C
:106BF000D8A46DD12751FE0DF3502A6B296F036A7B
:106C000027516F0FE96E020E0320EA6E036AEF5000
:106C10002925016E2A5103220150710FE96E010EE0
:106C20000320EA6EEF6A2751FE0DF3502A6B296F9D
:106C3000710E2925016E010E2A21036E01C02BF36E
:106C40002C6F2E6F01C02DF3010E306F540E2F6F7D
:106C50000001A4EC22F002C024F301C023F30301DD
:106C6000235303E12453D8B4F2D02E6B2D6B010EC5
:106C7000306F540E2F6F0001A4EC22F002C026F3F7
:106C800001C025F30301255303E12653D8B4DFD017
:106C900024C32AF323C329F3010E2C6F580E2B6F44
:106CA0000001FCEC22F001520FE024C32AF323C3BD
:106CB00029F3010E03012C6F5C0E2B6F0001FCEC1D
:106CC00022F00152D8A48ED026C32EF325C32DF373
:106CD000010E0301306F560E2F6F0001A4EC22F05D
:106CE00002C026F301C025F326C33DF325C33CF3C0
:106CF000D3EC25F003012751040DF350036A710F03
:106D0000016E020E032201C029F303C02AF326C339
:106D10002CF325C32BF30001CEEF26F02AC3EAFFA4
:106D200029C3E9FF00C0EFFF01C0ECFF02C0ECFF88
:106D300003C0ECFF03012E6B2D6B010E306F560E5E
:106D40002F6F0001A4EC22F002C026F301C025F34E
:106D500003012551261121E02751040DF350036A48
:106D6000710FE96E020E0320EA6EEFCF29F3ECCF2C
:106D70002AF3ECCF2BF3ECCF2CF32CC334F32BC33F
:106D800033F32AC332F329C331F326C336F325C3C1
:106D900035F300019CEC28F0030124C32AF323C33C
:106DA00029F3010E2C6F580E2B6F0001FCEC22F022
:106DB00001520CE1036A03012751700FE96E020EC4
:106DC0000320EA6E010EEF6E0BD00001036A03018F
:106DD0002751700FE96E020E0320EA6E020EEF6E6D
:106DE00035D00001036A03012751700FE96E020ECE
:106DF0000320EA6EEF522AE024C32AF323C329F3C7
:106E0000010E2C6F610E2B6F0001FCEC22F0015281
:106E10001CE1D89003012735036A750F016E020E3D
:106E2000032201C029F303C02AF326C32CF325C390
:106E30002BF30001F0EF28F02AC3EAFF29C3E9FF92
:106E400002C0ECFFED5201C0EFFF030138D0036A2E
:106E500027516F0FE96E020E0320EA6EEF522FE109
:106E6000036A2751700FE96E020E0320EA6EEF509D
:106E700002080FE1D8902735036A220FE96E010E50
:106E80000320EA6E010EEC6EED52040EEF6E2183CC
:106E900013D0D8902735036A220FE96E010E032024
:106EA000EA6E010EEC6EED52060EEF6E28C32CF367
:106EB0000001E4EC29F0030100010BD00301036A97
:106EC00027516F0FE96E020E0320EA6EEF6A50D66B
:106ED00000019AEC14F002C02AF301C029F3D89003
:106EE00003012735036A770FE96E020E0320EA6E6D
:106EF000ECCF03F0ED52EFCF01F00250035C04E35E
:106F000005E10150295D02E3000E01D0010E036A84
:106F1000031021E0D8902735036A770FE96E020E3F
:106F20000320EA6EECCF03F0ED52EF50FF08296F1B
:106F3000FF0E03542A6F00019AEC14F00150030174
:106F4000292702502A23010E2925016E000E2A212D
:106F5000036E01501AD000019AEC14F002C02AF31B
:106F600001C029F3D89003012735036A770FE96E32
:106F7000020E0320EA6EECCF03F0ED52EF50015CFD
:106F8000006E03500258036E0050C8081AE22751E1
:106F9000040DF350036A710FE96E020E0320EA6ECE
:106FA000EF68EC68EC68EC68D8902735036A220F2C
:106FB000E96E010E0320EA6E010EEC6EED52060E34
:106FC000EF6E21B303D00001FCD203010001D89081
:106FD00003012735036A220FE96E010E0320EA6ED2
:106FE000010EEC6EED52050EEF6ED8902735036A58
:106FF000770F016E020E032201C029F303C02AF3AA
:1070000000019AEC14F02AC3EAFF29C3E9FF02C089
:10701000ECFFED5201C0EFFF036A030127516F0F30
:10702000E96E020E0320EA6EEF6A000128C329F31D
:107030009FEC21F00152D8B4DFD028C329F3030E0E
:1070400003012B6F220E2A6F0001B5EC21F00152D3
:10705000D8B4D2D0D89003012735036A750FE96EF2
:10706000020E0320EA6EECCF2AF3ED52EFCF29F3A4
:10707000295305E12A53D8A402D00001BDD0D890ED
:107080002735036A750FE96E020E0320EA6E010EC2
:10709000EF5C006E000EEC58036E0050ED52EF6E88
:1070A00003C0ECFF225126081BE02751FE0DF350D0
:1070B0002A6B296F036A27516F0FE96E020E0320B6
:1070C000EA6EEF50EF2A036A2925016E2A51032246
:1070D0000150710FE96E010E0320EA6E22C3EFFF2B
:1070E0002251260812E0D8902735036A750FE96E01
:1070F000020E0320EA6EECCF2AF3ED52EFCF29F314
:107100002953D8A477D02A5375E12751FE0DF350A7
:107110002A6B296F036A27516F0FE96E020E032055
:10712000EA6E036AEF502925016E2A5103220150AD
:10713000710FE96E010E0320EA6EEF6A2751040D0C
:10714000F350036A710FE96E020E0320EA6EEFCF6F
:1071500029F3ECCF2AF3ECCF2BF3ECCF2CF3275110
:10716000FE0DF3502E6B2D6F710E2D25016E010E4D
:107170002E21036E01C02FF3306F2CC334F32BC3C9
:1071800033F32AC332F329C331F3366F01C035F329
:1071900000019CEC28F0D89003012735036A750F95
:1071A000E96E020E0320EA6EECCF2AF3ED52EFCF28
:1071B00029F3295317E12A5315E1D8902735036A9B
:1071C000220FE96E010E0320EA6E010EEC6EED5205
:1071D000060EEF6E28C32CF30001E4EC29F00CD06E
:1071E0000AD00301036A27516F0FE96E020E0320D4
:1071F000EA6EEF6A00011AD79AEC14F002C02AF383
:1072000001C029F3D89003012735036A770FE96E8F
:10721000020E0320EA6EECCF03F0ED52EFCF01F047
:107220000250035C04E305E10150295D02E3000E16
:1072300001D0010E036A031021E0D8902735036ABC
:10724000770FE96E020E0320EA6EECCF03F0ED52E9
:10725000EF50FF08296FFF0E03542A6F00019AECCC
:1072600014F001500301292702502A23010E292579
:10727000016E000E2A21036E01501AD000019AEC13
:1072800014F002C02AF301C029F3D8900301273576
:10729000036A770FE96E020E0320EA6EECCF03F06B
:1072A000ED52EF50015C006E03500258036E005027
:1072B000C8081AE22751040DF350036A710FE96EF2
:1072C000020E0320EA6EEF68EC68EC68EC68D89078
:1072D0002735036A220FE96E010E0320EA6E010EC4
:1072E000EC6EED52060EEF6E00016BD103012751DB
:1072F000040DF350036A250FE96E010E0320EA6EB8
:10730000EE52EE52EC6AED52EF6AED52EF6AED5238
:10731000EF6AD8902735036A220FE96E010E032029
:10732000EA6E010EEC6EED52070EEF6E000128C3FF
:107330002CF3E4EC29F028C34CF30BEC2AF00152B7
:10734000D8B49AD003012751040DF350036A710F8A
:10735000E96E020E0320EA6EEFCF29F3ECCF2AF399
:10736000ECCF2BF3ECCF2CF3293D22D02A3D20D0BB
:107370002B3D1ED02C3D1CD0010E036E1E0E296F1E
:1073800003C02AF327C32DF3010E2F6FF40E2E6FC7
:10739000336B326B03C031F329C330F3356B346B7D
:1073A000000152EC32F00301219101B0218154D04F
:1073B0002751040DF350036A710FE96E020E03208A
:1073C000EA6EEF5206E1EC5204E1EC5202E1EC52BB
:1073D00028E02751040DF350036A710FE96E020E85
:1073E0000320EA6EEFCF29F3ECCF2AF3ECCF2BF397
:1073F000ECCF2CF327C32DF32F6BC80E2E6F2CC3AD
:1074000033F32BC332F32AC331F329C330F3356B83
:10741000346B000152EC32F00301219101B0218163
:107420001BD0000E036EDA0E296F03C02AF327C3A8
:107430002DF3010E2F6F940E2E6F336B326B03C042
:1074400031F329C330F3356B346B000152EC32F069
:107450000301219101B0218121A10DD0D8902735C0
:10746000036A220FE96E010E0320EA6E010EEC6E34
:10747000ED52080EEF6E0001A4D0D890030127351D
:10748000036A220FE96E010E0320EA6E010EEC6E14
:10749000ED52090EEF6ED8902735036A770F016E13
:1074A000020E032201C029F303C02AF300019AEC63
:1074B00014F02AC3EAFF29C3E9FF02C0ECFFED5232
:1074C00001C0EFFF28C32CF3E4EC29F028C34CF3F0
:1074D0000BEC2AF001525FE19AEC14F002C02AF39F
:1074E00001C029F3D89003012735036A770FE96EAD
:1074F000020E0320EA6EECCF03F0ED52EFCF01F065
:107500000250035C04E305E10150295D02E3000E33
:1075100001D0010E036A031021E0D8902735036AD9
:10752000770FE96E020E0320EA6EECCF03F0ED5206
:10753000EF50FF08296FFF0E03542A6F00019AECE9
:1075400014F001500301292702502A23010E292596
:10755000016E000E2A21036E01501AD000019AEC30
:1075600014F002C02AF301C029F3D8900301273593
:10757000036A770FE96E020E0320EA6EECCF03F088
:10758000ED52EF50015C006E03500258036E005044
:10759000320813E2000128C329F313EF34F0D89026
:1075A00003012735036A220FE96E010E0320EA6EFC
:1075B000010EEC6EED520A0EEF6E000102D00301D7
:1075C00000010301272BB4EF34F00001CFEF3BF0B3
:1075D00003012091209102017951F90FD8B0D7D041
:1075E000070F0001D1EF3BF0020E0301226F7A0E6C
:1075F000216F030E246F1F0E236F0001F6EF0AF0B8
:10760000015203E10201C3D00001030120811F5395
:1076100005E1020E0201796F0DD003011F5106082A
:1076200005E1050E0201796F05D00301000183EC2D
:107630000AF00201ACD054EF0FF0015203E0020156
:10764000796B00010201A3D0030E0301226F1B0E10
:10765000216F020E246F7A0E236F030E266F1F0E0A
:10766000256F020E286F840E276F0001CEEF10F0F9
:10767000015219E0030120811F2D05D0030E0201E4
:10768000796F0FD003011F51060805E1060E0201B4
:10769000796F07D003012091000183EC0AF0020109
:1076A000796B05D0000183EC0AF00201796B6FD091
:1076B000020E0301226F7A0E216F030E246F1B0E40
:1076C000236F85C226F384C225F30001F6EF1CF078
:1076D000015203E00201796B0001020158D002015E
:1076E000796B855329E18451480826E3020E030192
:1076F000226F840E216F030E246F1F0E236F020E64
:10770000266F860E256F22C328F321C327F3020EAE
:107710002A6FC60E296F020E2C6FC80E2B6F000148
:107720003DEF1EF001520AE003011F51080805E178
:107730002081040E0201796F0301000183EC0AF03D
:10774000020125D0010E0301AA6F000128EC15F0FB
:1077500001521AE0020E0301226F7A0E216F236B91
:10776000020E256F860E246F84C226F3C7C228F34B
:10777000C6C227F3C9C22AF3C8C229F30001AAEF7F
:107780001EF00201796B0001020101D00201030128
:1077900020B120D7000135EF1FF0B2EF34F00BEF2E
:1077A0003DF0E824F76AF736BD0FF66E770EF72244
:1077B0000A00F550FA6E0800F550F96EE875E875A4
:1077C0004876DE7644773676B076F86AD09E078EB5
:1077D000536A526A546A556A5D6A5C6A040E606F45
:1077E0005F6A0201F76BFB6BFA6BF96BF86BFC6B72
:1077F0000301066B056BC150C00B0F09C16E070E6C
:10780000B46E5A9244D002004B000001005E000AA0
:107810004117000380FE000129412B001C8020003D
:107820003F0047455400504F535400436F6E7465FA
:107830006E742D4C656E6774683AFFC0000BC00013
:10784000464284000402CD4500002004C000188098
:1078500064112A9D0A0B0C0D0A0B0C0E0400040186
:1078600000080000010203040AC0000802FD2F0006
:107870002F6A736F6E0014030764657631006970B8
:107880006774006970006D696E74656D0000000EAC
:10789000F86E780EF76E060EF66E0900F550006E63
:1078A000000A13E00900F550016EE8BE05D00F0B89
:1078B000EA6E0900F5CFE9FF01BC090001AC09003F
:1078C000F5CFEEFF004EE9D7F9D7F86AC150C00BEB
:1078D0000F09C16EC290C66A070EB46E9250926EC6
:1078E000140E006E002EFED70000B450A19CCF6A8B
:1078F000830ECE6E030ECD6E9D80C00EF21200017F
:1079000078EF05F085EF05F078EF0AF0196AF2BE1E
:10791000198EF29E0A0E0301E16F00015EEC03F086
:1079200019BEF28E196AF2BE198EF29ECC0E0301B8
:10793000E16F00013CEC03F019BEF28E196AF2BE51
:10794000198EF29E4E0E0301E16F00013CEC03F034
:1079500019BEF28E196AF2BE198EF29E7D0E0301D7
:10796000E16F00013CEC03F019BEF28E196AF2BE21
:10797000198EF29EC90E0301E16F00013CEC03F089
:1079800019BEF28E196AF2BE198EF29E7F0E0301A5
:10799000E16F00013CEC03F019BEF28E196AF2BEF1
:1079A000198EF29E23EC03F019BEF28E196AF2BE14
:1079B000198EF29ECC0E0301E16F00013CEC03F046
:1079C00019BEF28E196AF2BE198EF29E480E03019C
:1079D000E16F00013CEC03F019BEF28E196AF2BEB1
:1079E000198EF29E0F0E0301E16F00015EEC03F0B1
:1079F00019BEF28E196AF2BE198EF29E6EEC04F078
:107A000019BEF28E03C0FBF202C0FAF201C0F9F215
:0A7A100000C0F8F2DDD5FED7030038
:020000040030CA
:0E00000007CC3E1E000781000FC00FE00F402E
:00000001FF
